:020000040000fa
:08104000ce570400000000007f
:020000040000fa
:10100000501a00000002000000050000000000006f
:020000040000fa
:10104800820e0400000000000058040000000000a8
:1010580006580400000000000c58040000000000be
:101068001258040000000000820e04000000000076
:10107800820e040000000000820e04000000000040
:10108800820e040000000000820e04000000000030
:10109800820e040000000000e221040000000000ad
:1010a800820e040000000000820e04000000000010
:1010b800820e040000000000145504000000000027
:1010c800820e040000000000820e040000000000f0
:1010d800820e040000000000820e040000000000e0
:1010e800820e040000000000241904000000000023
:1010f800820e040000000000820e040000000000c0
:10110800820e040000000000820e040000000000af
:10111800820e040000000000465604000000000093
:10112800820e040000000000820e0400000000008f
:10113800820e040000000000820e0400000000007f
:10114800820e040000000000820e0400000000006f
:10115800820e040000000000820e0400000000005f
:101168000a56040000000000820e0400000000007f
:10117800820e040000000000820e0400000000003f
:10118800820e040000000000820e0400000000002f
:10119800820e040000000000820e0400000000001f
:1011a800820e040000000000820e0400000000000f
:1011b800820e040000000000820e040000000000ff
:1011c800820e040000000000820e040000000000ef
:1011d800820e040000000000820e040000000000df
:1011e800820e040000000000820e040000000000cf
:1011f800820e040000000000820e040000000000bf
:10120800820e040000000000820e040000000000ae
:10121800820e040000000000820e0400000000009e
:10122800820e040000000000820e0400000000008e
:10123800820e040000000000820e0400000000007e
:10124800820e040000000000820e0400000000006e
:10125800820e040000000000820e0400000000005e
:10126800820e040000000000820e0400000000004e
:10127800820e040000000000820e0400000000003e
:10128800820e040000000000820e0400000000002e
:10129800820e040000000000820e0400000000001e
:1012a800820e040000000000820e0400000000000e
:1012b800820e040000000000820e040000000000fe
:1012c800820e040000000000820e040000000000ee
:1012d800820e040000000000820e040000000000de
:1012e800820e040000000000820e040000000000ce
:1012f800820e040000000000820e040000000000be
:10130800820e040000000000820e040000000000ad
:10131800820e040000000000820e0400000000009d
:10132800820e040000000000820e0400000000008d
:101338008855040000000000820e04000000000030
:10134800820e040000000000820e0400000000006d
:10135800820e040000000000820e0400000000005d
:10136800820e040000000000820e0400000000004d
:10137800820e040000000000820e0400000000003d
:10138800820e040000000000820e0400000000002d
:10139800820e040000000000820e0400000000001d
:1013a800820e040000000000820e0400000000000d
:1013b800820e040000000000820e040000000000fd
:1013c800820e040000000000820e040000000000ed
:1013d800820e040000000000820e040000000000dd
:1013e800820e040000000000820e040000000000cd
:1013f800820e040000000000820e040000000000bd
:10140800820e040000000000820e040000000000ac
:10141800820e040000000000820e0400000000009c
:10142800820e040000000000820e0400000000008c
:020000040000fa
:10160000001b04000000000003f0a200889fbe0041
:101610008a9fbe008c1f7800320107003901330019
:101620006450e1004f0032006420e10052003200bb
:1016300003826c0007003b000905d0000306d000c0
:10164000820f54000c065d000200390002003200d7
:1016500089017800030678008582550004003d006a
:101660000003fd008103fd008502ea008b85420036
:10167000840f720002003b0060001000e080180040
:101680006011b8000005eb007a28e1000a0039007b
:1016900006007800c75ddd00f707b200878075009f
:1016a0002d003700828171000a0178006105600019
:1016b0008180d1000080d3008502e900f9ff3b0062
:1016c000060440008784480002003b0060041400c8
:1016d000e0841c000988a300070032008a817100a1
:1016e00082817100610164008904d1000884d30003
:1016f0008b05e800170037000978a30013003a00b3
:101700000b00e000130034008b05e90008044400de
:1017100089844c000a4474000978a3000d003a0043
:101720000b00e000070034008b05e90008044400ca
:1017300089844c0001003a000b0020000978a300c6
:10174000f7ff32000001eb000200370082817100d8
:101750000a017800a80007000cf0a70001f0a00023
:10176000f10037006420e10002003a00838f6c0032
:10177000f10033000801be000200be00ea0037009d
:10178000889fbe008a9fbe008c1f7800d50007008e
:10179000dc00330003866c006450e1002e00320050
:1017a0006420e100330032006150e1002f0032007c
:1017b0006120e1003100320085855500eb07b00063
:1017c0000900200008042000050037000804440038
:1017d00089844c000a0031000603430087834b00d4
:1017e0000001530081815b00f8ff33000203be005b
:1017f0000800a0000804440089844c00f6ff39006a
:10180000c639dd008301730001003200130020009f
:101810008904d1000884d3000998a3000500320090
:101820000800a7000300a0008904d1000884d300a9
:101830008b05e8008904d1000884d3000001eb0087
:101840000281d2006c00070001f0a1000cf0a7009b
:1018500001f0a000b40037006420e100b6003200bf
:101860000801be000200be00f7ff37006120e10062
:10187000b10032006000b800f3ff37000000200024
:1018800001f82700f0ff3700839f68000100e000a7
:1018900002003d0060001000e08018000300e0003e
:1018a00002003d0060011100e0811900d90007002d
:1018b0004f00e00002003b0060001000e0801800d4
:1018c0000000060014002000e5003700f4ff2f00a0
:1018d000e30037000001be006d0007000470a700a0
:1018e00003f0a10003f8a30013003a006509b1005a
:1018f00010003200090035006928e10002003500bf
:101900000100280000000500000040008180480020
:101910008502e900fcff3a0000000600f88f420053
:10192000050035008100d1000080d3008502e80069
:10193000fcff3a00000006008000eb0000000500fc
:10194000881f7800010478000100e00005003d00d8
:1019500060001000e080180002003b0001f02c0045
:10196000030037000400070008f0a70001f0a00002
:101970004f04780000000600889fbe008a9fbe00ca
:10198000010578000000e000180032000004be00ed
:101990006011b8006b0920000982cf0002003900f5
:1019a0000882cf000441b000694252000e003200ac
:1019b00008003b0082817100610164008904d1004c
:1019c0000884d3008b05e8000442e800f9ff3a00e0
:1019d000050037000804440089844c008b05e900a9
:1019e0000442e900fbff3a00030007004f05be0078
:1019f0004f04be00000006008100200061805500f9
:101a00000b003d000b00200061fe2f000100e100f3
:101a10001d00340082817100610164008904d100dd
:101a20000884d3000000e800faff3a0071002000ab
:101a300061006400030070000200600009003200d1
:101a400061044400e0844c000988a50005003200d0
:101a50008b05e8006808e10002003a008904d10023
:101a60000884d300f20f20000258e10005003d0079
:101a7000c75ddd00f907b2008980750008007800b5
:101a8000000006000bf827008b007800000005001e
:101a9000c70ade00f107b200f50fb20008003200fd
:101aa000e1cf4200020032000170a00024000500d6
:101ab000810f700001003200040805004400050099
:101ac000810f700002003a00140005008502e90051
:101ad0000000400081c04800fcff3b000170a000f6
:101ae000240005000004be00e9ff07000003be005b
:101af0000405be000200be00e5ff0700844f75002c
:101b0000000006000200be006450e100050036003f
:101b10006420e100020036000968a30001003a00d9
:101b20000800be000160a0004f0678004f05be000f
:101b30004f04be0000000600f0ff2f00f1ff270059
:101b4000f9ff3700889fbe008a9fbe008c1f780077
:101b5000e4ff0700ebff330003866c006450e100f4
:101b6000240032006420e100270032006150e100cf
:101b7000220032006120e100210032008b8542000a
:101b8000eb07b1000134b800003ab8000804420085
:101b900089844a00013ab8000030b80088804000cb
:101ba00009014a0004003300000040008180480021
:101bb000020149008b05e900c909dd0083017000bd
:101bc0000100320013002000c814de004814dd00bc
:101bd0004709de001200b200c808de000884700069
:101be00085ff070001f0a1000cf0a70001f0a000a4
:101bf000cdff37006120e100cfff32000801be00b9
:101c00000200be00f7ff37006150e100fcff3a0020
:101c1000c9ff37006022b800060220000000d00093
:101c20008180d2000482d2008582d2000000a00010
:101c30000202520083825a00030031000202420075
:101c400083824a000000a1000603e900f3ff3a0086
:101c500000000600efff07000400be0000000600c1
:101c6000889fbe008a9fbe00841f78009dff0700ea
:101c70004f00780011003300f0ff2f00838f6c00bd
:101c800006003b00040565000a00a70008003700b5
:101c900009f0a6001000200008003700820f540051
:101ca000838f5c00030039001000200001003e001b
:101cb0000000200009f0a7000000ea004f05be0068
:101cc0004f04be000000e000000006008001780024
:101cd00002003700b15978000201e900e00f51001d
:101ce000fcff3a0000000600800178000200370087
:101cf000815978000201e900e00f5100fcff3a0031
:101d0000000006000040da000000fe000200fa00b9
:101d100012000700004f78009e4078000040eb0062
:101d200080cf50000200320084000700faff370025
:101d3000cd42a800cd62a90060d823000100200098
:101d40000a010700cd42a900cd62a90060d8230096
:101d50000100200005010700efff37000400fa0032
:101d600010c0b300004f7800900280001007980068
:101d7000ff3ffc0011028000f0f12f0000806000a6
:101d8000100288001e009000900288000000880069
:101d9000a0ff2000e07f880006120700203023000b
:101da000103a88000000eb00203a8800220007006b
:101db00053000700609d220001002000eb00070097
:101dc000680007002a1007000b0107003701070011
:101dd000c60007000000eb0072000700d7050700ef
:101de0008040eb00814f500002003a000040eb00c1
:101df000004f7800090607008040eb00814f50003b
:101e000002003a000040eb00004f78009e030700fc
:101e10009e4078000040eb0080cf5000020032006e
:101e2000cd42a900cd62a900221207001e40780011
:101e30000080fa00000006000000fa0020ff2f00da
:101e400060198800c922a900c962a900c942a90075
:101e5000cd22a800cd42a800cd62a800e862a9006a
:101e6000e042a900ec62a900e442a900e862a800ef
:101e7000e402a800d842a900e002a900e422a800d8
:101e8000e022a900cc22a900dcc2a900c822a90036
:101e9000d8c2a900d862a800d882a900d842a80058
:101ea000dc82a900da42a900e4a2a900cca2a90020
:101eb000cc82a900e0a2a900e0c2a900c8a2a900a2
:101ec000c882a900e4e2a800e462a900e662a800d2
:101ed000e0e2a900e062a900c862a800c842a80028
:101ee000d8c2a900c822a900d942a900d922a900b4
:101ef000c9c2a900d822a9000080fa00000006008b
:101f00000000fa00420020008000eb0040ff2000ab
:101f100075ff07000040eb00f4efb70020c0b300ee
:101f2000f5efb7000040eb00f6efb70050c0b3008c
:101f3000f7efb7000080fa00000006000000fa008a
:101f400002003700f11107004f06070045050700a2
:101f50008040eb00814f5000faff3a000080fa0009
:101f6000000006000000fa0000e0200000038800e6
:101f70000000eb00100388008660a9006105800066
:101f8000f0ff2800808060000000210000807000c9
:101f9000600588006340a8009660a8000080fa00f1
:101fa000000006000200fa00000f78009e00780092
:101fb0000000eb00808f500003003a00e4e2a8002c
:101fc000e462a80002003700e4e2a800e462a9008d
:101fd0000080fa00000006000a00fa00008fbe0030
:101fe0002207980033079800440798000000eb0090
:101ff000000988000000eb00f00888001e61a800be
:102000003e009000a07588004e009000c0758800ca
:102010002e009000b07588001e01be000024240030
:10202000f1002000800f5100818f59001000360010
:102030001e00be004206200003002000f5fe07003f
:10204000026420000289b900020178006002b90030
:102050008401780003014100036420000300b800fc
:102060000101410082007800008fbe000f003700a0
:102070001e00be00026420000289b900020178003f
:102080006002b9008401780003014100036420006c
:102090000300b800010141008200780042062000e0
:1020a00003002000dbfe0700008fbe000e0078005a
:1020b0000080e80010007800e00888000e0078003a
:1020c00010007800d00888008780a9009105800062
:1020d00080ff2f00008060000000a00090058800b5
:1020e0009780a8000080fa00000006000000fa00b7
:1020f000000320008008880084e0a900c0142500a7
:102100006008880031058000f0ff280080806000b2
:1021100000002200008070003005880094e0a800d4
:102120000080fa00000006000000fa0011e1a8009b
:102130000080fa00000006000000fa000000eb003a
:10214000c00888000000eb00a00888008780a90074
:102150001fe1a8000080fa00000006000000fa005d
:102160001fe1a9000080fa00000006000400fa0048
:10217000008fbe001e01be006000b800800f51003d
:10218000818f59001a003200f4ff07001e01be00c3
:102190002001200001002000800f5100818f590094
:1021a00004003600e0fe2f00f1ff2f001e0f40005c
:1021b0005e9748000002eb008001eb000001eb009d
:1021c0001e00be0084ff07009780a900daff070009
:1021d00000000000310480000000210080806000c9
:1021e0000000eb00808f5000faff32008780a900ca
:1021f0000080fa00000006000200fa00020220003f
:102200008000eb00a0eb2000b7fe0700a0eb200051
:1022100004000700004f78001e4078000080fa009c
:10222000000006000400fa001007980010c0b30078
:10223000004f78001e009000e40020000500200000
:10224000000178004000200001002000130f07006b
:10225000004f78001e009000104078001047980052
:102260009e40900000c0eb0080cf5000080032007c
:102270009e4090000040eb0080cf500004003200f0
:102280009e4078000040eb0080cf500004003a00f0
:10229000d2002000c14f2d00a0eb20008bfe0700d4
:1022a0001e4078000080fa00000006000200fa00dc
:1022b000020220008000eb00a0ed20008afe070053
:1022c000a0ed200004000700004f78001e407800b9
:1022d0000080fa00000006000400fa0010079800d1
:1022e00010c0b300004f78001e00900004022000d0
:1022f000050020000001780060012000010020009e
:10230000e60e0700004f78001e0090001040780095
:10231000104798009e40900030c2b30080cf50001c
:1023200004003a009e4078000040eb0080cf50004f
:1023300002003a000040eb00004f78001e40780099
:102340000080fa00000006000600fa00000f780086
:1023500011079800220798001e007800ae00900038
:102360000108bb001e0078009e0090000188bb00a1
:102370000080fa00000006000000fa0010002400af
:10238000003b880050052000303b8800a00a200058
:10239000303b880061e7a80000000000000000005a
:1023a00000000000013b80000000280080806000e9
:1023b0000000eb00808f5000faff3a000080fa0026
:1023c000000006001000fa006007980071079800ee
:1023d000100280004500de00674060000080fb00c6
:1023e0005007980090028000000f7800ff3ffc002b
:1023f00011028000f0f12f0080806000000c2000ae
:1024000000807000100288001e0078009002880092
:1024100000008800e07f80008000eb000108780069
:102420006e009000fe0090004008de0001002000d9
:10243000100798006e0090002007980032c0bf007f
:102440000080fb00300798001e00900000407800dc
:1024500032e0b70020042400003b88002e009000ea
:10246000ae0090000108bb0050052000303b880002
:10247000a00a2000303b880061e7a80000000000af
:102480000000000000000000013b80000000280068
:10249000808060000000eb00808f5000faff3a005f
:1024a0003e0090000040780032e0b700e07f8000fe
:1024b0003100200001087800900280004007980059
:1024c000ff3ffc005e009000004078006740600025
:1024d0000080fb00670060004500dd001202800004
:1024e000f1f12f008100610000807000100288006f
:1024f0004e00900090028800000088000080fa00e2
:10250000000006001800fa00100f9800220f980033
:10251000330f9800100280004500de006740600025
:102520000080fb00000f98009002800020079800b8
:10253000ff3ffc0011028000f0f12f00808060005e
:10254000000c200000807000100288002e00900017
:102550009002880000008800e07f80008000eb008f
:10256000010878002e089000be0890004008de00a8
:1025700001002000300798002e08900010079800f6
:1025800032c0bf000080fb00400798003e00900072
:102590000040780032e0b7000000eb00000f780048
:1025a000200037001e089000104078000080fb00db
:1025b000500798001e0890000000e800100f9800d7
:1025c0001e089000104078000080fb004800dd00ed
:1025d000de00900000807000500798001e089000f8
:1025e0000000e800100f98001e08900010407800ce
:1025f0000080fb00600798001e0890000000e800c3
:10260000100f98005e019000ee0090001e009000f8
:102610004dff07001e0090000080e80010079800a2
:102620001e0fe800f00320009e007800808f50000d
:10263000dcff360050ff07004e009000004078009d
:1026400032e0b700e07f8000310020000108780010
:102650009002800070079800ff3ffc000e08900079
:1026600000407800674060000080fb006700600069
:102670004500dd0012028000f1f12f0081006100b1
:1026800000807000100288007e0090009002880098
:10269000000088000080fa00000006000000fa0038
:1026a00000002a002100200046ff0700f0ceb30002
:1026b000faeeb700e0cbb300fbeeb7000040eb0052
:1026c000fceeb70002002a0023002000a0ef20004b
:1026d0008cff07000080fa00000006000c00fa00e2
:1026e0000040eb00004f78006800470052a88600c9
:1026f00063a886000288be0034c0bf000080fb00d3
:102700001007980010c0b30034e0b70000002f009d
:10271000200798002e009000900178003307980061
:10272000be009000a0992a00808f500019003a0046
:102730002e0090000080e800420020008000780019
:10274000a0fb200061fd070068004700ae0090007c
:102750008180e8001001780090019000110078005d
:10276000910090003f000700004f78009e407800e5
:1027700010c0b30080cf500003003a000d000700e6
:10278000004f7800050037000040eb00004f780054
:10279000020037000040eb00004f78001e00900060
:1027a0000040780034e0b7001e4078000080fa0056
:1027b000000006000a00fa000040eb00004f78001d
:1027c00050c0b30034e0b70000ff290010079800a4
:1027d0001e0090009000780021079800ae00900045
:1027e000a0992a00808f50001b003a001e00900024
:1027f0008080e800660047004200200033fd0700ab
:102800006600470090409000bbcfbf0080cf5000d3
:1028100011003a0066004700a0409000bccfbf0006
:1028200080cf50000c003a0066004700b040900096
:10283000bdcfbf0080cf500007003a0066004700c0
:1028400090407800bacfbf0080cf500002003a001d
:1028500010c0b300004f78001e4078000080fa00de
:10286000000006000a00fa000e82e800000a780064
:1028700011029800660047000208780013009800d3
:102880000040eb00004f78000e80e8009040900080
:10289000660047001040900080cf50001e003e00b0
:1028a0000e80e800904090006600470010409000c5
:1028b00080cf500006003a000e80e800a040900053
:1028c000660047002040900080cf500012003e007c
:1028d0000e80e80090409000660047001040900095
:1028e00080cf500019003a000e80e800a040900010
:1028f000660047002040900080cf500013003a004f
:102900000e80e800b0409000660047003040900024
:1029100080cf50000d0039000e80e8009040780014
:10292000660047001040780080cf5000050031005d
:1029300066004700904078000040eb0080cf5000d8
:1029400002003a0010c0b300004f78001e4078002b
:102950000080fa00000006000200fa00004f780034
:102960009e4078000040eb0080cf50000200320013
:10297000ec22a80001003700ec22a900e822a900ff
:102980000080fa00000006000000fa00ff0b0900ba
:10299000000000000080fa00000006000400fa00b9
:1029a00095a0a90085a0a9000000eb0000198800ef
:1029b0000000eb00401988000000eb00801988003f
:1029c00000102000201988000000eb00101988007a
:1029d00021e3a800ecff07000000eb0010079800bf
:1029e0000000eb00000f7800100037002023a80043
:1029f000e5ff07002023a900000000000019800067
:102a0000e10060000000eb00808f5000fbff32000f
:102a10009e0078000018800000804000000f7800c1
:102a20001e0090000000e800100798009e00900033
:102a3000f0002000808f5000ecff34009e007800f2
:102a40000000eb00808f50000c0032001e00780068
:102a5000cf80de00bafb070002002000031824002c
:102a600047fb07000001be00000020000102240017
:102a700043fb070040868800518688000000eb0079
:102a8000001988000080fa00000006000000fa002b
:102a90000000eb0000198800203020004019880059
:102aa00050002000101988004002210020198800e1
:102ab000000e20000019880085a0a90095a0a9009b
:102ac00051058000f0f82f00808060000006200093
:102ad00000807000500588002043a80021e3a80072
:102ae000800c200001002000a0fd07000080fa00fb
:102af000000006000200fa0095a0a9006086800090
:102b0000000f780095a0a8001e0078000080fa0051
:102b1000000006000200fa0095a0a900908680003f
:102b2000000f780095a0a8001e0078000080fa0031
:102b3000000006000a00fa00881f7800300798009d
:102b4000410798000200200003e023003e009000af
:102b5000ce0090000afb07005efb0700000f780024
:102b60001e0078000100200083fb07000200200007
:102b700003e02300f3fb07000001be003e009000cd
:102b8000ce009000a0fa07001007980021079800d7
:102b900018c0b3000200200003d823001e009000dc
:102ba000ae00900049fb07008000eb00810f500051
:102bb00001003c000044eb000040eb00804f54005b
:102bc000010032001e0fe8001e0078004f0478005c
:102bd0000080fa00000006000400fa00c5ff0700ac
:102be0000100200064fb07000002be004086800058
:102bf000518680000001be000400be00d1fb07002a
:102c0000d27d2a0083eb2300ddfa0700008fbe008f
:102c10001e00be000080fa00000006000400fa005a
:102c2000bcff07000100200053fb07000002be00ac
:102c300040868000518680000001be000400be0076
:102c4000c0fb0700127e2a0083e32300ccfa0700b2
:102c5000008fbe001e00be000080fa0000000600cb
:102c60000000fa00dcff0700b2ff07000080fa0056
:102c7000000006000000fa00e8ff0700adff0700b3
:102c80000080fa00000006000000fa00c2012000e7
:102c90008000eb00800c210013fc0700ec62a9000f
:102ca000e442a900e862a900e042a9000000eb00ac
:102cb00090088800900620007008880013e1a800a2
:102cc00036ff070071ff0700e230a8001000200067
:102cd000f08688000040eb00b4010700c00020002f
:102ce000a0000700c00020001e0007000080fa00be
:102cf000000006000400fa00004f78001107980059
:102d00009e4078000040eb0080cf50000b003a005e
:102d10000000eb00d00c88000000eb00000d8800e4
:102d20001e009000f00c8800d0002000e00c88000d
:102d300070402000d00c8800080037000000eb0035
:102d4000800c88000000eb00b00c88001e00900092
:102d5000a00c8800d0002000900c88000080fa00b1
:102d6000000006000800fa00300798000040eb0061
:102d7000004f78003e00900001002000fefa07009e
:102d80000200200003e023006efb070010079800fc
:102d9000210798001e009000ae009000050007007b
:102da00010c0b300004f78001e4078000080fa0089
:102db000000006000a00fa00881f7800300798001b
:102dc0004107980010c0b300004f780095a0a900fb
:102dd00051058000f0f82f00808060000006200080
:102de0000080700050058800e2f0a900e310a900ff
:102df000e2b0a90018c0b3000200200003162400ae
:102e00003e009000ce009000b0fa07008000eb007a
:102e1000810f500001003c000044eb000040eb003b
:102e2000804f5400060032000000200001162400ec
:102e300030079800410798000040eb00004f7800f1
:102e40006011b8003e009000ce0090009dfa07008f
:102e50008000eb00810f50000b003a000000eb00f7
:102e6000800c8800118780000004200080806000b2
:102e70000000eb00808f50000100320095a0a800f8
:102e800010c0b300340037003233230033f3230083
:102e90003e009000ce0090002afb0700100798002b
:102ea0002107980095a0a900127e2a0083e3230041
:102eb0001e009000ae00900022fb07000002be0042
:102ec00040868000518680000001be000400be00e4
:102ed0002bfa07007ffa070000007800a086880020
:102ee0000000eb00b086880050052000e0868800d6
:102ef000127e2a0083e323003e009000ce00900063
:102f000010fb07000002be00408680005186800052
:102f10000001be000400be0019fa070002002000f4
:102f200003082400b9f907006afa070000007800d6
:102f3000c0868800c086800068005000d086880067
:102f40005105200010c0b3006aff0700e310a8007d
:102f500095a0a8001e4078004f0478000080fa0079
:102f6000000006000c00fa00881f78005007980047
:102f70000040eb00004f78005e0090000100200050
:102f80007dfa07000200200003e02300edfa0700ad
:102f900010079800210798001e009000ae009000d6
:102fa000450007000cff0700300798004107980014
:102fb0002bff07004087880040878000308788000b
:102fc0001e019000ae0190003e009000ce009000e7
:102fd0008df9070001f0a10018c0b300a2702d0008
:102fe00033e2230037fa07008000eb00810f500026
:102ff000010035000044eb000040eb00804f54001e
:103000000300320010c0b300004f78000100370009
:10301000000000001e4078004f0478000080fa0095
:10302000000006000a00fa00881f780030079800a8
:10303000410798000040eb00004f78003e009000f0
:10304000ce0090001c000700e3fe07001007980068
:10305000210798003e019000ce0190001e009000d4
:10306000ae00900068f9070001f0a10018c0b3009d
:10307000a2702d0033e2230012fa07008000eb005b
:10308000810f5000010035000044eb000040eb00d0
:10309000804f54000300320010c0b300004f78008e
:1030a00001003700000000001e4078004f04780047
:1030b0000080fa00000006000a00fa00881f78006d
:1030c000300798004107980010c0b300004f780007
:1030d00095a0a900e2d0a9006011b8003e009000c0
:1030e000ce009000f7f907008000eb00810f500040
:1030f00004003a000000eb00d00c880010c0b300c0
:103100004e00370018c0b30002002000030a24005c
:103110003e009000ce009000ecf907008000eb002c
:10312000810f500001003c000044eb000040eb0028
:10313000804f54000600320000002000010a2400e5
:1031400030079800410798000040eb00004f7800de
:10315000a299290093f523003e009000ce00900034
:1031600078fa0700100798002107980018c0b300ec
:10317000a2702d00330824001e009000ae009000c5
:10318000d2f907008000eb00810f500001003c00e5
:103190000044eb000040eb00804f5400040032007c
:1031a000a0702d0031082400100798002107980016
:1031b000d27d2a0083eb23001e009000ae00900019
:1031c00060fa07000002be00408680005186800041
:1031d0000001be000400be0069f90700bdf9070048
:1031e00000007800708688000000eb008086880070
:1031f000f2282c0053d723003e009000ce00900010
:103200005ff907000200200003f02300fff8070029
:10321000b0f9070000007800800078000040eb0063
:10322000b4fe0700e2d0a80095a0a800007122001b
:1032300001002000cdfb07001e4078004f047800fd
:103240000080fa0000000600809fbe00821f780008
:103250000800fa00100280004500de0067406000b0
:103260000080fb003007980090028000000f78007b
:10327000ff3ffc0011028000f0f12f008080600011
:10328000000c200000807000100288001e007800f2
:103290009002880000008800e07f80008000eb0042
:1032a0000108780034c0bf000080fb0010079800c0
:1032b000000020000040780034e0b70085a0a9009d
:1032c00000188000608688001018800090868800b2
:1032d0001187800000082000808060000000eb0063
:1032e000808f5000160032001187800000022000fd
:1032f000808060000000eb00808f500010003a00da
:1033000091868000c0868000808f500002003600c9
:103310000000eb00800c880091868000d086800041
:10332000808f500006003100810c80000000eb000f
:10333000808f500002003a0070402000800c88000e
:103340001e0090000040780034e0b700e07f80006d
:1033500031002000010878009002800020079800ca
:10336000ff3ffc003e009000004078006740600096
:103370000080fb00670060004500dd001202800055
:10338000f1f12f00810061000080700010028800c0
:103390002e00900090028800000088000080fa0053
:1033a0004f0178004f00be00004006000200fa0006
:1033b000004f78009e4078000040eb0080cf500026
:1033c0000f00320011878000001020008080600014
:1033d0000000eb00808f500006003200704020009b
:1033e000800c8800e2f0a800801a2600010020006e
:1033f0005efb0700e4c2a900e4a2a80011003700a8
:103400001187800000022000808060000000eb0037
:10341000808f500009003a00e2f0a9000000eb00a4
:10342000800c8800e4c2a80080b5210001002000c3
:103430004efb0700e4a2a90002003700e4a2a900a5
:10344000e4c2a8000080fa00000006000000fa00b4
:10345000201780004500de00614060000080fa0017
:10346000000006000000fa00da0107008000ea0010
:10347000008070004f00de00004078000080fa00fd
:10348000000006000600fa00000f780012079800fe
:10349000230798001e019000ae0190001e007800e6
:1034a000fb0107001e0090001e0040000080fa0093
:1034b000000006000200fa001200200003002000b5
:1034c0000e007800f20107001e4078000080fa002c
:1034d000000006000000fa0010c0b30050e8b7007a
:1034e0006000b80090428800a14288000040eb00d4
:1034f0005ae8b7000040eb005be8b7000040eb0083
:103500005ce8b70010c0b3005de8b7006000b80029
:10351000b0428800c14288000080fa000000060026
:103520000000fa000000eb00004588000000eb00fe
:10353000104588000080fa00000006001e00fa0016
:10354000426120008000eb00008a2000e6f90700bd
:10355000e0ff0700f2ff07000000eb00000f78001b
:103560001a003700a1ed20009140780030c2b3006e
:1035700080cf50000b003a009e00e800a0ed200034
:1035800000804000104078008080fb000e81e80041
:103590001e00780000004000000041000108780093
:1035a00009003700a0eb20001e004000104078000a
:1035b0008080fb000e81e8001e00780000004000c3
:1035c00000004100010878001e0fe8009e0078000e
:1035d000d0002000808f5000e2ff34009b060700df
:1035e0000e80e800b8060700de03070010c0b30035
:1035f000a5e8b70010c0b3000080fa000000060084
:103600000200fa00000f78009e00780010c0b3009e
:10361000804878000080fa00000006000400fa00ec
:103620000040eb00004f78000040eb00204798007e
:103630000040eb00104798000e80e8000002780080
:1036400003b021000001eb00006c2c00d10220002f
:1036500061fa0700b8fa070010003700fd03070001
:10366000210321009140780000c2b30080cf5000b8
:1036700004003200ae4090000040eb0080cf5000cc
:103680000600320010c0b300004f780010c0b30035
:103690001047980010c0b300affc07009e407800b0
:1036a0000040eb0080cf5000ecff32009e409000c5
:1036b0000040eb0080cf5000090032009ec0a900fe
:1036c0008ec0a90071068000f08f2f0080806000fe
:1036d0000060200000807000700688009ec0a80076
:1036e00010c0b3000080fa00000006000800fa00d5
:1036f000000f780012079800230798006147980090
:1037000000000000e80007008040eb00814f5000ff
:10371000fcff32009e0078000000eb00808f50001c
:103720000e003a001e019000c07f800090007800db
:1037300013458000808a20000080410063f9070063
:10374000c07f8000c17f8000110178009e00900042
:103750008100410001087800070037009e009000ba
:1037600012458000808a200000004100010178009d
:103770009e00780055f90700114580001e0090005a
:103780000080400010458800014580001e00900028
:103790000080400000458800ee4090000040eb00b3
:1037a00080cf500001003200370007000080fa008f
:1037b000000006000000fa000080fa000000060089
:1037c0000800fa00100798002207980033079800b5
:1037d000ae00900012458000808a20000000410069
:1037e000010178009e00900038f907000145800033
:1037f0002e00900000804000004588000000eb0093
:10380000000f7800090037001e007800e800400033
:10381000008a20000080400010407800818a20004b
:103820009e804000804878001e0fe800f0032000d2
:103830009e007800808f5000f3ff36000045800026
:1038400000458800114580002e0090000080400057
:1038500010458800014580002e0090000080400047
:103860000045880003c4b300828a200011c0b30061
:1038700010c0b3007d0807008087880028ff07007c
:103880000080fa00000006000600fa00808a20008e
:10389000000f7800014580000000eb00808f500091
:1038a00045003200e1ff2000914078000040eb002d
:1038b00080cf50000300320080382100010020003a
:1038c0002afa07000000eb00200798000c003700e0
:1038d0002e009000e8004000008a20000080400098
:1038e000104078002e019000818a20008100410064
:1038f000804878002e0090000000e8002007980023
:10390000ae009000f0032000808f5000f0ff3600e2
:103910000045800000458800220037008187800034
:103920000000eb00808f5000050032000000000016
:10393000960007008040eb00814f5000fcff3200f2
:103940000145800000042000808f500003003600f5
:1039500000c4b300204798000200370000458000f3
:1039600020479800014580002e4090000080fb0019
:10397000008050000045880003c4b3001e01780099
:1039800011c0b30010c0b30038080700808788005a
:103990002e4090000080fb001e0f40000040eb0016
:1039a000a5e8b700014580000000eb00808f5000c3
:1039b000daff3a00dafe07000080fa000000060095
:1039c0000000fa0000000000718780000000eb009a
:1039d000808f5000080032007087800090007800cf
:1039e00000002800808060000000eb00808f500005
:1039f000f5ff3a00010037000000000081878000d9
:103a00000000eb00808f50000700320080878000ac
:103a10009000780000002800808060000000eb002b
:103a2000808f5000f5ff3a00006a28001100200046
:103a3000cef907000000eb00a02488000000eb0096
:103a4000602488000040eb0032f0b7000080fa00ec
:103a5000000006000200fa00000f78002103210098
:103a60009140780000c2b30000c068000080fb00f5
:103a70000000e9004f00de00004078000080fa00fe
:103a8000000006000600fa00004f780012079800b8
:103a9000230798000080fa00000006000000fa00ea
:103aa0000080fa00000006000000fa00a5c8bf0070
:103ab0000080fa00000006000000fa0010c0b30009
:103ac0000080fa00000006000800fa0010028000e2
:103ad0004500de00674060000080fb003007980072
:103ae00090028000000f7800ff3ffc001102800070
:103af000f0f12f0080806000000c2000008070003a
:103b0000100288001e0078009002880000008800e3
:103b1000e07f80008000eb00010878005ac8bf00f9
:103b20000080fb000000ea004f00de002047980004
:103b3000e07f8000310020000108780090028000c2
:103b400020079800ff3ffc003e00900000407800f6
:103b5000674060000080fb00670060004500dd00fa
:103b600012028000f1f12f008100610000807000de
:103b7000100288002e00900090028800000088004b
:103b80002e4090000080fa00000006000000fa00bd
:103b9000818780000000eb00808f5000070032001a
:103ba00080878000900078000000280080806000fe
:103bb0000000eb00808f500002003a00100020004f
:103bc000010037000000eb00004078000080fa00a0
:103bd000000006000800fa00100280004500de0028
:103be000674060000080fb00300798009002800072
:103bf000000f7800ff3ffc0011028000f0f12f0061
:103c000080806000000c200000807000100288009e
:103c10001e0078009002880000008800e07f80008d
:103c20008000eb00010878005ac8bf000080fb004c
:103c300010079800e07f8000310020000108780024
:103c40009002800020079800ff3ffc003e0090009b
:103c500000407800674060000080fb006700600063
:103c60004500dd0012028000f1f12f0081006100ab
:103c700000807000100288002e00900090028800e2
:103c8000000088001e0090000080fa00000006007e
:103c90001a00fa00200f9800320f9800430f980086
:103ca0006000b80010079800210798000040eb0062
:103cb000004f78001b013700c6ff070060479800df
:103cc000ee4090000040eb0080cf5000e200320058
:103cd000100280004500de00674060000080fb00ad
:103ce000100f98009002800040079800ff3ffc00f2
:103cf00011028000f0f12f0080806000000c200095
:103d000000807000100288004e0090009002880031
:103d100000008800e07f80008000eb000108780050
:103d20006e4090000081fb00030020001e00900008
:103d3000ae00900002014000838148003e089000e0
:103d4000ce089000800f5100818f59004300390048
:103d5000ae0890000000eb00808f500013003a0086
:103d6000be0890001e009000008150005bc8bf009c
:103d70008080fb00e085200080804000c07f8000c4
:103d800010007800d1f70700c07f8000c17f80005d
:103d900011017800be0990009e00900081805100c2
:103da00081004100010878000b003700be08900038
:103db0001e009000808050005bc8bf000081fb00a7
:103dc000e0852000000041000101780080007800bb
:103dd0002e089000bdf70700b185200091407800c3
:103de0003e089000004178001e00900000407800de
:103df0000040510000c040005be8b700a1852000f2
:103e0000914078001e009000004178003e0890002c
:103e1000004078000040510000c040005ae8b70060
:103e2000b2428000c34280003e0a9000ce0a900059
:103e30001e009000ae0090000000520081805a00e9
:103e40000200400083804800b0428800c1428800e0
:103e500010c0b300004f780040003700ae0890005b
:103e60000000eb00808f500011003a006e4090007f
:103e70000081fb005bc8bf008080fb00e085200064
:103e800080804000c07f8000100078008ff707001e
:103e9000c17f8000c07f8000100178006e409000dc
:103ea0000080fb0000004100800878000f00370010
:103eb0006e4090008080fb005bc8bf000081fb006b
:103ec000e0852000000041000101780080007800ba
:103ed0002e0890007df707006e4090000080fb00e8
:103ee000ae08900000804000200f9800b1852000af
:103ef000914078006e40900000c040005be8b70041
:103f0000a1852000914078006e40900000c05000d4
:103f10005ae8b700b2428000c34280006e40900071
:103f20000080fb0001002000020040008380480068
:103f3000b0428800c14288006e4090000080fb00c3
:103f4000010020001e019000ae0190000200400020
:103f50008380480010079800210798009242800053
:103f6000a3428000b0428000c1428000800f510017
:103f7000818f590013003a006000b8009042880019
:103f8000a14288000040eb005ae8b7000040eb0077
:103f90005be8b7006000b800b0428800c14288000a
:103fa00010c0b3005de8b70003c4b300e285200091
:103fb0008040eb0010c0b300ac060700708788009b
:103fc00011003700b18520009140780000c4b30093
:103fd00080cf50000c003a000040eb005be8b700d7
:103fe0000040eb005ae8b70010c0b3005de8b7002e
:103ff00003c4b300e28520008040eb0010c0b30092
:104000009a06070070878800e07f8000310020005a
:10401000010878009002800050079800ff3ffc00e4
:104020001e08900000407800674060000080fb00a0
:10403000670060004500dd0012028000f1f12f00f2
:104040008100610000807000100288005e00900016
:104050009002880000008800100280004500de0009
:10406000674060000080fb00000f98009002800015
:1040700060079800ff3ffc0011028000f0f12f0064
:1040800080806000000c200000807000100288001a
:104090006e0090009002880000008800e07f8000a1
:1040a0008000eb0001087800c18520009140780075
:1040b0000040eb0080cf500006003200d185200088
:1040c000914078000040eb0080cf500001003200aa
:1040d00048000700e07f80003100200001087800e0
:1040e0009002800070079800ff3ffc000e089000cf
:1040f00000407800674060000080fb0067006000bf
:104100004500dd0012028000f1f12f008100610006
:1041100000807000100288007e00900090028800ed
:10412000000088009e4078000040eb0080cf5000e7
:10413000e1fe32000080fa00000006000800fa00ec
:104140000000eb00000f7800100280004500de0048
:10415000674060000080fb003007980090028000fc
:1041600010079800ff3ffc0011028000f0f12f00c3
:1041700080806000000c2000008070001002880029
:104180001e0090009002880000008800e07f800000
:104190008000eb0001087800e07f80003100200003
:1041a000010878009002800020079800ff3ffc0083
:1041b0003e00900000407800674060000080fb00f7
:1041c000670060004500dd0012028000f1f12f0061
:1041d0008100610000807000100288002e009000b5
:1041e00090028800000088001e0078000080fa001d
:1041f000000006000200fa000185200091407800ce
:104200000040eb0080cf50002c0032000004200062
:104210000100200090428800a14288000004200094
:10422000000f7800080037001e007800ee00400004
:10423000008520000080400010407800e1852000cb
:104240009e804000804878001e00ea001e0070003a
:104250004f00de00804078001e0fe9000040eb00b8
:1042600080cf5000f0ff3a000040eb005be8b70061
:1042700092428000a3428000000420000100200040
:10428000800f5100818f59000500360000c4b30033
:104290005ae8b7000040eb0050e8b70023003700b1
:1042a00090428000a1428000004078005ae8b700a8
:1042b00010c0b30050e8b7001c0037000040eb000e
:1042c0005be8b700b2428000c342800000042000d7
:1042d00001002000020140008381480090428000dc
:1042e000a1428000800f5100818f59000b003900de
:1042f00090428000a142800000417800b0428000de
:10430000c142800000407800004051005ae8b700e8
:1043100010c0b30050e8b7000400370000c4b30079
:104320005ae8b7000040eb0050e8b7000080fa0000
:10433000000006000000fa0055d0bf008080fb009e
:10434000b0ff2f008080600080012000808f50002f
:104350000a003a000040eb00a6e8b700418a2000be
:10436000914078000040eb0080cf500013003a00ed
:1043700010c0b300a5e8b7001000370055d0bf004b
:104380008080fb00b0ff2f008080600000012000d3
:10439000808f500009003a00d185200091407800bc
:1043a0000040eb0080cf50000200320091ff070078
:1043b0000200370010c0b3005ce8b7000080fa00cc
:1043c00000000600809fbe00821f78000800fa00ef
:1043d000100280004500de00674060000080fb00a6
:1043e0003007980090028000000f7800ff3ffc002b
:1043f00011028000f0f12f0080806000000c20008e
:1044000000807000100288001e0078009002880072
:1044100000008800e07f80008000eb000108780049
:1044200034c0bf000080fb0010079800000020008f
:104430000040780034e0b7008460a9001e009000be
:104440000040780034e0b700e07f800031002000b9
:10445000010878009002800020079800ff3ffc00d0
:104460003e00900000407800674060000080fb0044
:10447000670060004500dd0012028000f1f12f00ae
:104480008100610000807000100288002e00900002
:1044900090028800000088000080fa004f01780038
:1044a0004f00be00004006000000fa000080fa0045
:1044b000000006000000fa000080fa00000006007c
:1044c0000000fa000080fa00000006000000fa0078
:1044d0000080fa00000006000000fa00b80507009e
:1044e0000080fa00000006000000fa000080fa00d8
:1044f000000006000000fa00d1c1b30010c0b300f4
:104500000105070003c4b300e28520008040eb00f2
:1045100010c0b30055050700708788000000eb004d
:10452000808788000080fa00000006000000fa0082
:104530009444a80080702000c0878800c087800055
:104540000000e900c0878800c18780000000eb0000
:10455000808f5000f9ff3a009444a9000080fa00cf
:10456000000006000200fa00f00f2000702488000e
:10457000f00f200050248800f009200080248800db
:10458000f0092000602488008804a80000002100b1
:104590004800de00c02488009424a8009424a900c8
:1045a0000000eb00b02488000040eb00004f7800d2
:1045b000080037009e4078000180fb00c200dd004b
:1045c00000002100008140006000b8000089be00aa
:1045d0001e4fe8009e40780070c0b30080cf5000ae
:1045e000f4ff3600d000200050258800030037007b
:1045f000a048200031c0b3006505070050248000aa
:10460000e80060000000eb00808f5000f8ff3a00e7
:104610000040eb0046f0b700a10421000040eb0091
:10462000a0409800a00421008000eb002100980029
:1046300094a4a90080002100f08188000040eb00d4
:1046400033f0b7000040eb0032f0b7000080fa0012
:10465000000006000200fa002103210091407800ca
:104660000040eb0080cf500011003a000000eb004a
:10467000a02488000000eb006024880001003700bf
:104680009404a800a0248000e10060000000eb007a
:10469000808f5000faff320010c0b30032f0b70034
:1046a00020002000302588000001200040258800df
:1046b000210321009140780010c0b30080cf50004a
:1046c00008003a00f00f2000502488000000eb00a2
:1046d000602488008c04a8008c84a80020c0b3004b
:1046e00032f0b70000248000f00060000000eb0012
:1046f000808f50000600320010248000f00060001f
:104700000000eb00808f500001003200990007008c
:1047100040248000e20060000000eb00808f500029
:104720006c003a0050248000e10060000000eb00c3
:10473000808f50001400320060248000e10060008f
:104740000000eb00808f50000f00320085ff070053
:1047500040c0b30032f0b700a005210010808800ef
:1047600080c0b30000f0b70001d0bf00634060001c
:1047700001f0b7001100210091407800c0c8b300db
:1047800000c0700001f0b70050248000f00060000d
:104790000000eb00808f5000060032006024800093
:1047a000f00060000000eb00808f5000010032003c
:1047b0006800070050248000e40060000000eb0067
:1047c000808f50000900320060248000e400600007
:1047d0000000eb00808f50000400320038ff07001b
:1047e000a048200021c0b300e90407005124800044
:1047f00000082000808060000000eb00808f5000e7
:1048000007003200612480000008200080806000e2
:104810000000eb00808f50000100320034000700e0
:1048200050248000e20060000000eb00808f500008
:104830000800320060248000e20060000000eb000d
:10484000808f50000300320020ff0700f00f20008f
:1048500070248800210321009140780030c0b3000b
:1048600080cf50001d00360060248000e80060000a
:104870000000eb00808f50001b0032000040eb0076
:10488000004f78000e00370050248000e8006000e0
:104890000000eb00808f5000120032009024800056
:1048a0000040780055f0b700a048200031c0b300a8
:1048b000b7040700370007009efe07001e4fe80000
:1048c0009e40780030c0b30080cf5000eeff36002d
:1048d0000500370000000000030037000000000062
:1048e00001003700000000000080fa000000060010
:1048f0000000fa0050258000e20060000000eb009c
:10490000808f50000e003200b081800090409000f7
:1049100000c8b30080cf500008003a00f08180004a
:104920009040900040c8b30080cf500003003a0090
:10493000b1818000c0c8b30090409800aa24a900ab
:10494000a048200071c0b300910407000080fa0065
:10495000000006000000fa008284a800a0482000a1
:1049600041c0b3008a040700cffe07000080fa00b0
:10497000000006000000fa00cefe07008284a900b5
:104980000048200041c0b300810407000080fa0005
:10499000000006000000fa0055d0bf008080fb0038
:1049a000b0ff2f00808060000000eb00808f50007f
:1049b0001b003a0055d0bf000080fb004200de0023
:1049c000004078000080fb00c200dd0000002100f4
:1049d00000804000b0818800b0818000c0818800e4
:1049e0008103210080032100104078000024a200f0
:1049f00080487800b08180009000780000c02300db
:104a00008080600000402300808f500002003a0048
:104a10000d0007000a0037002300070008003700d8
:104a200055d0bf008080fb00b0ff2f008080600069
:104a300080002000808f500001003a002500070010
:104a40000080fa00000006000000fa00f0818000fb
:104a50009000780000002800808060000000eb00db
:104a6000808f500003003200f18180000040eb0095
:104a7000904098000040eb0042f0b7000040eb008f
:104a800043f0b7000000eb00408288000040eb00dc
:104a900046f0b700ac0007008ffe070038020700a1
:104aa0000080fa00000006000000fa003104210036
:104ab0009140780020c0b30080cf500002003a003f
:104ac000f302070001003700400007000080fa00f1
:104ad000000006000200fa00f0818000100078005b
:104ae0004e00de0061406000004f7800e1032100cd
:104af000e0032100104078000024a20080487800e4
:104b0000210321009140780080c0b30080cf500085
:104b10000d003a00a0052100204090000080fb001d
:104b2000b0248800b12480000000eb00808f50008a
:104b30000300320000c1b30032f0b70002003700ba
:104b400040c0b30032f0b70031042100914078003a
:104b500010c0b30080cf500019003a00f0818000ef
:104b6000210621001100980078020700210421008d
:104b70009140780020c0b30080cf500004003a007c
:104b8000f181800040c8b300904098000d003700cc
:104b90009e4078000040eb0080cf500004003a00b7
:104ba000f181800080ccb300904098000500370070
:104bb000f181800080c8b300904098000100370068
:104bc000020007000080fa00000006000400fa005e
:104bd000310421009140780020c0b30080cf500004
:104be0002f003a00a1248000000220008080600095
:104bf0000000eb00808f500029003200b08180005f
:104c00009040780080c0b30080cf500024003a006c
:104c1000b08180009000780000c023008080600098
:104c200000402300808f50001d003a00c0818000aa
:104c30009000780000002800808060000000eb00f9
:104c4000808f500016003a00c0818000a10521002d
:104c5000110098000040eb00004f78000b00370077
:104c60001e4078008080fb00a0052100808040006d
:104c70001e4078000081fb0020062100000041005a
:104c800010407800804878001e4fe8009e40780071
:104c900070c0b30080cf5000f1ff36001400370021
:104ca0000040eb0043f0b700c181800080c0b3003a
:104cb00080487800c0818000a10521001100980083
:104cc000c1818000c0c8b30090409800f18180008d
:104cd0000040eb0090409800f08180000020a2008e
:104ce000100798009e0090000040eb009040980054
:104cf000a004210090009000000820008080600047
:104d00000000eb00808f50000d003200a004210055
:104d1000b00090000000eb00808f500003003200d4
:104d2000a00421003000900000000100a004210038
:104d300010019000f1f72f00810061001100980030
:104d40000080fa00000006000000fa00a005210023
:104d50009000780000062000808060000000eb00da
:104d6000808f500040003a00a005210010409000c4
:104d70000080fb00cf80de00b20020000300200096
:104d8000820f5000838f580039003e000060010000
:104d90001a0037001b0037003700370019003700b2
:104da0003500370006003700090037002c003700b7
:104db0000b00370008003700140037001e003700d2
:104dc00046f0a80080c0b30032f0b7002b003700d7
:104dd000d5000700290037008202070027003700ae
:104de00030032100208288004610a80010c0b300c4
:104df00048f0b70046f0a800200037001501070072
:104e00001e0037001f0007001c003700a00521000e
:104e1000404090008080fb00400321000080400063
:104e2000208288004610a80010c0b30048f0b700e8
:104e300046f0a8001100370046f0a800a0052100a8
:104e4000404090000081fb00a00521002040900020
:104e500041032100810041008048780007003700ad
:104e6000a1fd070005003700000000000300370027
:104e70000000000001003700000000000080fa0080
:104e8000000006000600fa00a0052100a0409000e6
:104e900010c0b30080cf500011003a00a0052100df
:104ea00010007800ff0060000000eb00808f5000d1
:104eb0000b003a0046f0a800a005210090409000a9
:104ec00030c0b30080cf500003003a0010c0b300e0
:104ed00054f0b700020037000040eb0054f0b70078
:104ee000a0052100a04090000040eb0080cf5000c2
:104ef00054003a00a005210010007800ff00600077
:104f000020002000808f50004e003a00a0052100b4
:104f100020009000ef0060000000eb00808f500048
:104f20004800320046f0a8000040eb00004f780037
:104f3000400037000000210010079800a005210064
:104f400020009000004078006f4060000080fb006f
:104f50000000400080007800a005210020009000a3
:104f60004700de00614060000080fb0000804000e0
:104f700000004000800078001e4178000280fb00a5
:104f8000008040004200dd009e0090000080400054
:104f900010079800a00521009040900030c0b30099
:104fa00080cf500004003a009e00900040c8b3003b
:104fb000904098001e003700a005210020009000be
:104fc000004078006f4060000080fb00000040005f
:104fd00080007800a04a2000008040002007980050
:104fe0002e00900090007800d0ff2f00808060009d
:104ff0002e00900001087800a0052100a00090007c
:1050000000082000808060000000eb00808f5000ce
:10501000040032009e00900000c4b300904098004d
:10502000030037009e00900080ccb30090409800b1
:105030001e4fe8009e40780010c0b30080cf5000a3
:10504000bcff36000080fa00000006000a00fa00eb
:10505000a00a210010079800d0a78600300798000a
:105060003e009000104078000080fb004007980050
:10507000d0a78600200798000000eb00000f780002
:105080000b0037002e009000104078009e0090002a
:10509000804878001e0090000000e800100798008b
:1050a0002e0090000000e800200798001e0fe80086
:1050b0004e0090009e007800808f5000f1ff390074
:1050c0000080fa00000006000400fa0010079800b3
:1050d0000040eb00004f78000d0037009e40780044
:1050e0000180fb009e009000910078000000e80025
:1050f00000014000a00a21000000410001087800e2
:105100001e0090000080e800100798001e4fe80085
:105110009e407800d0c0b30080cf5000efff360033
:105120000080fa00000006000000fa00a00521003f
:105130009040780000c8b30080cf500043003a0090
:1051400000ccb30046f0b700a0052100304090002d
:105150000080fb0021002000810f50000b00320076
:1051600031002000810f5000160032001100200095
:10517000810f500032003a0000432d002082880049
:10518000200120004082880030003700a005210067
:10519000204090000080fb0000004000800078006c
:1051a000204f2d00008040001000780020828800f1
:1051b000208280000080e800100078004082880093
:1051c00022003700a0052100a040900030c0b300ad
:1051d00080cf50000c003a0046d0bf0046f0b70028
:1051e00046d0bf000004a00046f0b700a00a21008e
:1051f0002082880020828000104078000080fb0020
:105200004082880011003700a00521002040900056
:105210000080fb000000400080007800404f2d001f
:1052200000804000100078002082880020828000ea
:10523000104078000080fb004082880003003700a7
:105240000040eb0046f0b700000000000080fa00cc
:10525000000006000200fa000040eb0062f0b70018
:105260000040eb0063f0b700a005210010007800bb
:10527000004078007f4060000080fb0011002000ab
:10528000810f50001000320021002000810f5000db
:105290000f0032008000eb00810f50002b003a001d
:1052a00046f0a800410521009140780010c0b300ed
:1052b00080cf500022003a0062d0bf000014a0004e
:1052c00062f0b7002100370046f0a8001f00370049
:1052d00046f0a80000002100000f7800a005210082
:1052e00020009000004078006f4060000080fb00cc
:1052f0000000400080007800a00521002000900000
:105300004700de00614060000080fb00008040003c
:105310004300dd001e0f40001e007800104090008a
:105320000080fb00e40060000000eb00808f500074
:105330000500320010c0b30062f0b7000300370070
:1053400000000000010037000000000031828000f2
:1053500000082000808060000000eb00808f50007b
:105360000500320020062100208288004610a80097
:1053700020c0b30048f0b7000080fa00000006002b
:105380000000fa0094a4a9003182800000082000e7
:10539000808060000000eb00808f500026003a0003
:1053a000a004210090009000000820008080600090
:1053b0000000eb00808f50001200320020c0b300cc
:1053c00043f0b700f18180000040eb008048780096
:1053d000f181800080ccb30090409800c1818000b2
:1053e00080c0b30080487800c08180002106210081
:1053f00011009800c181800080ccb30090409800db
:1054000050003700c181800080c0b3008048780020
:10541000c0818000a105210011009800c181800099
:10542000c0c8b30090409800f181800040c8b3002c
:105430009040980043003700a004210090009000a5
:1054400000082000808060000000eb00808f50008a
:105450003c003a00a00521009000780000082000e0
:10546000808060000000eb00808f5000240032003c
:10547000a0052100b000900040828000808f500085
:1054800003003100a0052100300090004082880018
:105490002e00070010c0b30043f0b700c1818000a8
:1054a00080c0b30080487800c0818000a105210041
:1054b00011009800c181800000c8b300904098009e
:1054c000b181800080c0b30080487800b081800046
:1054d000a105210011009800b181800000c8b3002f
:1054e00090409800f0818000210621001100980072
:1054f000f181800080ccb30090409800110037000b
:1055000020c0b30043f0b700f18180000040eb0001
:1055100080487800f181800080ccb30090409800f2
:10552000c181800080c0b30080487800c0818000c5
:105530002106210011009800c181800080ccb300b9
:10554000904098000080fa00000006000200fa0077
:105550004182800070002000808f500012003e00c9
:1055600040828000000f78002104210091407800e3
:105570000040eb0080cf500003003a0010c0b300a1
:1055800042f0b7000a003700210421009140780062
:1055900010c0b30080cf500005003a0020c0b30017
:1055a00042f0b7000200370080002000000f7800b2
:1055b000f2818000f0818000904090001e409000b9
:1055c00000c0700010419800f18180001e407800fa
:1055d00080487800418280001e00780000805000e2
:1055e000408288002006210090828800308280005e
:1055f000e10060000000eb00808f50001d003a00c9
:105600000b003700928280002182800011407800d8
:10561000004978000200e800908288000100e8005c
:10562000208288001e0078000000e900000f78004a
:105630009e0078000000eb00808f5000f1ff3a00e0
:105640001100370092828000218280001140780092
:10565000004978000200e800908288000100e8001c
:10566000208288001e0078000000e900000f78000a
:1056700001003700000000009e0078000000eb00f1
:10568000808f5000efff3a000080fa000000060013
:105690000200fa00b0818000104f78001e407800b0
:1056a0008080fb00a004210020009000808f50002b
:1056b00004003600a004210020009000004f780074
:1056c00007003700a0042100a00090001e417800d0
:1056d0000280fb0080805000a0042100210098007f
:1056e0000040eb00104798000e003700a004210096
:1056f000900078001e4090000081fb0020062100f1
:105700000000410010407800804878008100e800e7
:10571000a0042100010878001e4090000040e8002d
:10572000104798009e4090001e40780080cf5000a7
:10573000eeff3900a0042100a00090000000eb0063
:10574000808f500015003200c181800080c0b300fe
:1057500080487800c0818000210621001100980057
:10576000b0818000900078000000240080806000fc
:105770000000eb00808f500004003a00c1818000df
:1057800080ccb3009040980014003700c1818000a5
:1057900080c8b3009040980010003700c08180009e
:1057a000a105210011009800a0042100b000900084
:1057b0000000eb00808f500003003200a0042100a5
:1057c0003000900000000100a004210010019000b2
:1057d000f1f72f0081006100110098000080fa00ad
:1057e000000006000000fa0046f0a80012002000a9
:1057f0008000eb00400321003bf10700a0052100e1
:105800002040900033f0b700a0052100a040900098
:105810000040eb0080cf500003003a0000c1b3000d
:1058200032f0b7000300370000c2b30032f0b70017
:1058300030fb07000080fa00000006000400fa00b8
:10584000204798003147980000002100000f7800a1
:105850002e4090000080fb00000040008000780097
:105860003e4090000080fb00008040004300dd00cf
:105870004200de004200dd001e0f40001e007800e6
:1058800010017800f1ff2700810061000108780015
:10589000be4090000040eb0080cf500007003a006f
:1058a0002e4090000080fb0080004000a0032100fb
:1058b000008040001e087800060037002e4090004f
:1058c0000080fb0080004000e003210000804000d9
:1058d0001e0878001e00780010017800f1ff2b00f0
:1058e00081006100010878009e007800648040001b
:1058f0001001780001002400810071000108780087
:105900000080fa00000006000400fa00204798001a
:10591000314798002e4090000080fb0000004000be
:1059200080007800a04a2000008f40003e40900098
:105930008080fb001e007800010878003e40900047
:105940000080fb00e80060000000eb00808f50004a
:10595000030032008040eb002e409000b7ff0700ac
:105960003e4090000080fb00e40060000000eb007f
:10597000808f50000300320011c0b3002e40900011
:10598000aeff07000080fa00000006000400fa00e5
:105990002047980031479800ae4090000040eb004f
:1059a00080cf50000d003a00c181800080c0b3005c
:1059b00080487800c0818000a10521001100980076
:1059c000c1818000c0c8b30090409800f181800080
:1059d00040c8b30090409800220037002e4090004d
:1059e0000080fb0000004000800078003e409000f6
:1059f0000080fb00008040004300dd008000780054
:105a000000002100008f40001e00780090409000b0
:105a100040c8b30000c070009e007800904098001d
:105a20002e4090000080fb000000400080007800c5
:105a30003e4090000080fb00008040004300dd00fd
:105a4000e400400000002100008f40001e007800ac
:105a50009040900040c8b30000c070009e007800e5
:105a6000904098000080fa00000006000800fa004c
:105a70002047980031479800220798006347980014
:105a8000be4090000040eb0080cf50000700320085
:105a90002e4090000080fb0080004000e0032100c9
:105aa00000804000100f7800060037002e40900064
:105ab0000080fb0080004000a00321000080400027
:105ac000100f78001e007800ae00900011009800c2
:105ad0001e007800ee409000014878001e0078001b
:105ae000104090000044b2009e0078009040980062
:105af0001e0078009040900080c8b30000c0700085
:105b00009e00780090409800be4090000040eb005e
:105b100080cf50000e003200e10321002e409000a3
:105b20000080fb000000400080804000e203210074
:105b30002e4090000080fb0000004000000041006b
:105b4000104078000024a200804878000d00370043
:105b5000a10321002e4090000080fb0000004000c7
:105b600080804000a20321002e4090000080fb00b6
:105b70000000400000004100104078000024a20016
:105b8000804878001e0078000080fa0000000600bf
:105b90000400fa00000f7800214798002e40900082
:105ba0000080fb00110020000008dd0000407800ac
:105bb0009e007800804878000080fa00000006000f
:105bc0000000fa00a005210010007800ff0060002e
:105bd00010002000808f500073003a00a0052100c3
:105be000c04090000040eb0080cf500070003a00b1
:105bf000a00521009040900060c0b30080cf50000d
:105c00002a003a00a0052100304090000080fb00ef
:105c100021022000810f50001200320031022000ca
:105c2000810f50001b00320011022000810f500034
:105c30001e003a00310321009140780010c0b300eb
:105c400080cf500016003a0040452d002082880089
:105c5000900020004082880000ccb30046f0b700de
:105c600012003700310321009140780010c0b300ca
:105c700080cf50000c003a00404d2d00208288005b
:105c8000d00120004082880000ccb30046f0b7006d
:105c90000600370000c8b30046f0b7000300370025
:105ca000000000000100370000000000a0052100f6
:105cb0009000780000062000808060000002200034
:105cc000808f50003c003a00a00521001040900059
:105cd0000080fb006101b9000080eb008080eb00d8
:105ce0000200400083804800a20020000300200042
:105cf000820f5000838f580030003e00006001008a
:105d00000a0037000d003700190037002b0037005c
:105d10002a00370029003700280037002700370005
:105d2000040037000c00370018003700250007007a
:105d3000220037002600070020003700200f210036
:105d400020828800100020004082880010ccb30020
:105d500046f0b7001900370000c8b30046f0b7009e
:105d6000a005210030409000f2f0b700130037008a
:105d7000300f21002082880010002000408288001f
:105d800010c8b30046f0b7000c00370000c8b300dd
:105d900046f0b700a005210020409000f3f0b700c6
:105da000000000000500370000000000030037007d
:105db0000000000001003700000000000080fa0031
:105dc000000006000000fa000080fa000000060053
:105dd0000000fa000080fa00000006000000fa004f
:105de0000080fa00000006000200fa00004f780070
:105df0000000eb00001388008820a9009820a9006b
:105e00009e4078000040eb0080cf5000030032003d
:105e1000b01320001013880002003700e0132000a8
:105e20001013880000002800001388000080fa008a
:105e3000000006000200fa00004f78009e40780043
:105e40000180fb0040138800000000000013800068
:105e5000e10060000000eb00808f5000fbff32008b
:105e600040138000004078000080fa000000060027
:105e70000000fa00d8a2a900dca2a800f122a90023
:105e8000f522a800d8e2a900dce2a800e802a900f7
:105e9000ec02a8000080fa00000006000c00fa00e6
:105ea00010079800210798003207980044079800cf
:105eb0005507980010c0b300104798001e009000ce
:105ec000ae0090000001be006000b800800f5100dd
:105ed000818f590003003d0000cfb300004f7800d0
:105ee0000200370010cfb300004f78000041eb00f4
:105ef00011c0b3001e407800f8000700104798005a
:105f00009e4090000040eb0080cf50002f003200f8
:105f100030c0b300c7ff07009e40780000cfb30039
:105f200080cf500004003a000e80e8000080e800b6
:105f300010407800bfff07000e80e8000000e80076
:105f400010407800bbff07000e80e800104078008a
:105f5000b8ff0700070037000040eb00b5ff07005f
:105f6000be009000804878003e0090000000e800ed
:105f700030079800ce0090005e0090000080700016
:105f80008000ea00008070004f00de0000427800d0
:105f90004e019000de0190000080eb008080eb005d
:105fa0000200400083804800400798005107980095
:105fb0000040eb00804f5200e7ff3a000041eb0049
:105fc0008040eb001e407800c40007001e40900097
:105fd0000080fa00000006001e00fa00889fbe0044
:105fe000200f9800310f9800420f9800540f98002e
:105ff000650f980010c0b300004f780010c0b300c8
:10600000104f98002e099000be0990006000b80063
:10601000800f5100818f59000b003d0000cfb3006d
:10602000604f980000102000100798000040eb001f
:10603000004f9800803e200001002000500798008b
:10604000610798000a00370010cfb300604f980036
:10605000000420001007980010c0b300004f980003
:10606000803e200001002000500798006107980042
:106070002e089000be089000000f9800110f9800a5
:106080007f0037001e0090006101b8005e0890009c
:10609000ee089000800f5100818f590003003e00f0
:1060a0009e00900021079800020037005e089000d3
:1060b000200798002e0090006101b8000e089000a3
:1060c0009e08900002024000838248001e0090005b
:1060d000010020000001be000400be00cdee07005c
:1060e0000004be000e0a90009e0a90001e00900060
:1060f000010020000001be000400be00c5ee070044
:10610000800f5400818f5c000f0032002e00900041
:106110006101b8000e0890009e0890000202400045
:10612000838248001e009000010020000001be0094
:106130000400be00c7ee070000007800ae0090002b
:1061400000805000200798009e4890000040eb001f
:1061500080cf5000030032000040eb00104f980049
:10616000050037005e019000ee0190006e4890003f
:10617000c4000700004f78009e4078000040eb000c
:1061800080cf50003e00320012c0b30011c0b300f7
:106190006e48900051000700004f78009e40780044
:1061a0000040eb0080cf50003500320020c0b3002b
:1061b00020ff07008e4890000040eb0080cf500089
:1061c00004003a00700047000080e80010407800aa
:1061d00018ff0700700047000000e800104078003a
:1061e00014ff0700700047001040780011ff0700ff
:1061f0000000eb0030079800090037004e089000bf
:1062000010407800ce0890008100e800410f98000f
:1062100008ff07003e0090000000e80030079800eb
:10622000be0090002e009000808f5000f3ff3900d8
:106230000041eb008040eb006e4890002700070013
:106240002e009000010020005e099000ee099000f1
:106250000000510081805900500f9800610f980094
:106260002e0090006101b8000e0890009e0890007a
:106270000200400083804800000f9800110f980032
:106280009e4078000040eb0080cf500006003200b6
:106290005e099000ee0990006000b800800f510088
:1062a000818f590077ff3a009e4078000040eb0054
:1062b00080cf5000050032005e019000ee0190009a
:1062c0006e4890006f000700004f78001e40780075
:1062d0004f04be000080fa00000006000600fa002d
:1062e00020479800314798004247980010c0b300fb
:1062f000004f78000040eb0010479800ae4090003f
:1063000000cfb30080cf500003003a0010c0b300ac
:106310001047980009003700ae40900010cfb3003e
:1063200080cf500003003a000040eb001047980077
:10633000020037000040eb00004f7800dca2a8000c
:10634000dce2a800f522a800ec02a8009e4078003c
:106350000040eb0080cf50002c003200be40900087
:106360000040eb0080cf5000280032009e4090009b
:106370000040eb0080cf50000900320010c0b30095
:1063800099fe0700f522a900ce4090000040eb00e6
:1063900080cf50000a003200ec02a800080037004d
:1063a0000040eb0090fe0700dca2a900ce40900068
:1063b0000040eb0080cf500001003200dce2a8007a
:1063c000ce4090000040eb0080cf50000f00320024
:1063d00060c0b30097fe07009e4090000040eb00b5
:1063e00080cf500005003200f522a8000000000018
:1063f00000000000f522a90004003700dca2a8007c
:106400000000000000000000dca2a9001e4078008f
:106410000080fa00000006000600fa0020479800fd
:10642000210798000040eb00004f78000041eb008e
:1064300011c0b3002e409000a8ff07008040eb0081
:10644000814f50000c00320050c0b30079fe0700ad
:106450000040eb0077fe0700ae0090008048780017
:1064600010c0b300004f78000041eb008040eb000b
:106470002e40900099ff07001e4078000080fa002f
:10648000000006000a00fa00404798003207980012
:10649000430798000040eb00004f780010c0b300a5
:1064a000104798000c0037000e80e800800078004c
:1064b0004e409000d8ff0700104798001e00900043
:1064c000e10060000000eb00808f500002003a0005
:1064d00010c0b300004f78009e4078000040eb00f1
:1064e00080cf500016003a00be0090004e00900091
:1064f000008070008000ea00008070004f00de0025
:10650000004278003e019000ce0190000080eb0038
:106510008080eb0002004000838048003007980034
:10652000410798000040eb00804f52000400320009
:106530009e4090000040eb0080cf5000daff3a0010
:106540003e019000ce0190006000b800800f510025
:10655000818f590002003a000040eb00104798007c
:106560001e4090000080fa00000006000000fa00c3
:106570002174200062042000730520008248780006
:106580008348780042c7a9000080fa000000060096
:106590000000fa002174200062042000730520002e
:1065a000824878008348780042c7a8000080fa003b
:1065b000000006000000fa00ecff070051368000e2
:1065c00000fc2f00008060003000b30050368800cf
:1065d0002135800000fc2f00008060001001b30016
:1065e00020358800c1368000f00f2c0080806000cc
:1065f0000070200000807000c0368800b136800036
:10660000f00f2c008080600000802000008070006f
:10661000b03688004135800000fc2f00008060000b
:106620006001b3004035880041358000f00f2c0038
:10663000808060000070210000807000403588007c
:1066400051368000f00f2c008080600000a02000f8
:1066500000807000503688001136800000fc2f004a
:1066600000806000b000b300103688006135800003
:1066700000fc2f0000806000c000b300603588007f
:106680009136800000fc2f00008060002001b300e4
:1066900090368800e136800000fc2f00008060000a
:1066a0003001b300e0368800b9ff07000080fa002f
:1066b000000006000000fa0000002400607f88004f
:1066c000607f8000707f8800607f80000030b000b5
:1066d000407f8800407f80000010b000507f88001d
:1066e000507f80000008b000807f8800807f80009d
:1066f0000004b000907f8800907f80000004b0000c
:10670000307f88000080fa00000006000400fa00d4
:106710000000eb0010079800807f8000020420003a
:106720000300200057f30700807f80009e00900048
:106730000100400010407800beefb7000100e80003
:1067400010079800becfbf000080fb006101b900b8
:10675000c0fd2f00f1ff2f000200400083804800a1
:106760006209200003002000820f5000838f580030
:1067700078013e0000600100a1003700750137007c
:10678000740137007301370072013700710137005f
:10679000a60037006f0137006e0137006d0137002a
:1067a0006c0137006b0137006a013700690137005f
:1067b000680137006701370066013700650137005f
:1067c000640137006301370062013700610137005f
:1067d000600137005f0137005e0137005d0137005f
:1067e0005c0137005b0137005a0137007900370040
:1067f0005b0137005701370056013700550137005c
:10680000540137005301370052013700510137005e
:10681000500137004f0137004e0137004d0137005e
:106820004c0137004b0137004a013700490137005e
:10683000480137004701370046013700450137005e
:10684000440137004301370042013700410137005e
:10685000430137003f0137003e0137003d0137005b
:106860003c0137003b0137003a013700390137005e
:10687000380137003701370036013700350137005e
:10688000340137003301370032013700310137005e
:10689000300137002f0137002e0137002d0137005e
:1068a0002c0137002b0137002a013700290137005e
:1068b000280137002701370026013700250137005e
:1068c000240137002301370022013700210137005e
:1068d000200137001f0137001e0137001d0137005e
:1068e0001c0137001b0137001a013700190137005e
:1068f000180137001701370016013700150137005e
:10690000140137001301370012013700110137005d
:10691000100137000f0137000e0137000d0137005d
:106920000c0137000b0137000a013700090137005d
:10693000080137000701370006013700050137005d
:10694000040137000301370002013700010137005d
:1069500000013700ff003700fe003700fd00370060
:10696000fc003700fb0037003b0037004d003700cc
:106970005f003700600037006100370063003700b8
:10698000700037008400370085003700870037002b
:1069900088003700890037008a003700e0003700a0
:1069a000dd00370089003700e6003700df003700e0
:1069b000e1003700ea003700e9003700e100370066
:1069c000e7003700e300370082003700c2003700dd
:1069d000cf003700817f80001e00900000804000c3
:1069e000904078000040eb0080cf500001003a005a
:1069f000ee0d07000004200010079800d9003700b2
:106a0000817f80001e009000008040009040780050
:106a10000040eb0080cf500001003a00140e070048
:106a20000004200010079800ce003700817f80000e
:106a30001e00900000804000904078000040eb0075
:106a400080cf500001003a002d0e07000004200006
:106a500010079800c3003700817f80001e0090005f
:106a600000804000104078008080fb00827f800022
:106a70001e0090000000e800000041001040780077
:106a80000080fb004800dd00008f40001e00780001
:106a900034f107001e0090000080e8001007980005
:106aa000b0003700817f80001e0090000080400011
:106ab000104078008080fb00827f80001e009000e4
:106ac0000000e80000004100104078000080fb005a
:106ad0004800dd00008f40001e007800a1f0070094
:106ae0001e0090000080e800100798009d0037000d
:106af000960707009b0037007504070099003700d0
:106b00000e80e800e307070096003700817f8000d1
:106b10001e0090000000e8000080400090407800d7
:106b2000827f80001e00900000004100104078002d
:106b30009d0807001e0090000080e80010079800e4
:106b400088003700817f80001e0090000080400098
:106b500010407800827f80009e0090008100e80055
:106b600001014100804078000200780083000700a6
:106b7000817f80001e00900000804000104078005f
:106b80008080fb001e009000008040000000e800b4
:106b90001007980073003700f508070071003700f0
:106ba0000e80e800fb0807006e0037003f04070076
:106bb0006c003700720507006a003700a307070062
:106bc000680037002809070066003700a2080700a0
:106bd00064003700807f80009e009000010040002c
:106be00010407800c9efb7000100e80010079800d6
:106bf000807f80009e0090000100400010407800df
:106c0000beefb7000100e80010079800807f800009
:106c10009e0090000100400010407800c0efb700d7
:106c20000100e80010079800807f80009e0090001f
:106c30000100400010407800c2efb7000100e800fa
:106c400010079800807f80009e00900001004000a7
:106c500010407800c3efb7000100e800100798006b
:106c6000807f80009e00900001004000104078006e
:106c7000c4efb7000100e80010079800807f800093
:106c80009e0090000100400010407800c5efb70062
:106c90000100e80010079800807f80009e009000af
:106ca0000100400010407800c8efb7000100e80084
:106cb00010079800807f80009e0090000100400037
:106cc00010407800caefb7000100e80010079800f4
:106cd0006e09070023003700817f80001e009000ae
:106ce0000000e8000080400090407800827f800033
:106cf0001e0090000000410010407800320a07009a
:106d00001e0090000080e800100798001500370072
:106d100000000000130037000000fe0011003700e3
:106d200000042000100798000e0037000e80e800d5
:106d3000800a07000b0037000e80e8003c0a0700bd
:106d4000080037001e009000640040001007980003
:106d500004003700000420001007980001003700ed
:106d6000000000009e009000f0032000808f500083
:106d70006dfe36000080fa00000006001000fa00e8
:106d8000889fbe008a1f780060079800614f9800b6
:106d90000040eb00004f78000040eb0020479800d7
:106da0000040eb00304798000040eb00404798005f
:106db0000000eb00300798000040eb00004f980007
:106dc0000040eb00104f9800ee4890000040eb00b0
:106dd00080cf500004003200ee489000d0c3b300d2
:106de00080cf50009f033600e1afa800ab0337000f
:106df0009e4078000180fb00ee0090000080400083
:106e000010407800beefb700e1fb20009140780011
:106e100010cbb30080cf500003003e006e499000bd
:106e2000024f780092033700becfbf000080fb0006
:106e30006101b900e0f42f00f1ff2f0002004000d3
:106e400083804800d204200003002000820f5000fd
:106e5000838f580085033e00006001000303370064
:106e6000ef013700f3013700f7013700fb0137006e
:106e7000fd013700090237002402370040023700c5
:106e800048023700500237005e02370073023700b5
:106e90007203370071033700700337006f03370048
:106ea0007e023700820237008b0237008f023700e4
:106eb000920237009a0237009e023700a202370082
:106ec000a5023700ad023700af023700b10237002c
:106ed000b4023700be023700ca023700da023700b8
:106ee000f9023700100337002a003700340037005a
:106ef0003800370045003700520037007100370076
:106f000087003700890037008c0037001f033700e7
:106f1000220337002a0337002d0337003b033700d5
:106f2000b5003700b7003700be003700d800370083
:106f3000f2003700fa00370002013700290137005c
:106f4000310137003a013700440137005001370062
:106f50006001370063013700670137006c013700bb
:106f60007601370080013700830137008601370042
:106f7000880137008a0137008f01370096013700fa
:106f8000980137009a0137009c0137009e013700b5
:106f9000a00137001e4fe8009e4178000380fb00ef
:106fa000ee00900000804000104078000080fb0060
:106fb000030407003c0407001e4fe8002c033700c1
:106fc0001e4fe80080002000fd0307003604070084
:106fd000270337001e4fe80041002000100020006a
:106fe0007d030700810020000000eb007a0307000a
:106ff00080002000f20307002b040700800020001f
:10700000ef03070028040700190337001e4fe800ac
:10701000410020000000eb006f030700810020000a
:107020000000eb006c030700810020000000eb0073
:1070300069030700810020000000eb0066030700e1
:107040000b0337001e4fe800410020000000eb005a
:10705000610307001e4278000480fb00ee009000f0
:1070600000804000104078000080fb001e4fe800c8
:1070700081002000580307009e4078000180fb003b
:10708000ee00900000804000104078000080fb007f
:107090001e4fe800810020004f0307001e417800ca
:1070a0000280fb00ee00900000804000104078005d
:1070b0000080fb001e4fe80081002000460307000f
:1070c000eb0237001e4fe800410020000000eb00fb
:1070d000410307009e4178000380fb00ee00900012
:1070e00000804000104078000080fb001e4fe80048
:1070f00081002000380307001e4278000480fb0056
:10710000ee00900000804000104078000080fb00fe
:107110001e4fe800810020002f030700d402370033
:10712000fd0307001e4fe800d1023700ed090700fc
:10713000dd0307001e4fe800cd0237009e48900097
:107140000040eb0080cf50000e0032003e00900067
:107150000000e90030079800be0090000000eb003e
:10716000808f500004003a000040eb00104f980060
:107170001ecfe800be0237004e409000004f78005e
:10718000bb0237009e4078000180fb000000e80051
:10719000ee00900000804000104078009e40780093
:1071a00000c0500040479800db0307000080fb0050
:1071b00030079800d80307000080fb004800dd007e
:1071c000be0090000080400030079800be00900094
:1071d0000000eb00808f500002003a001ecfe80054
:1071e000a302370010c0b300104f98004e4190002a
:1071f000024f78009e023700ee499000034f78005e
:107200009b0237001e4278000480fb000000e8006b
:10721000ee00900000804000104078001e4f4000bb
:1072200093023700517f8000e2cfbf000080fb0057
:107230000000e9000080400090407800114798006d
:107240001e4178000280fb000000e800ee00900084
:1072500000804000904078001e40900080cf500099
:10726000080031009e4178000380fb000080e800a8
:10727000ee00900000804000104078001e4f40005b
:107280007b0237001e427800634f420078023700cd
:10729000517f8000e2cfbf000080fb000000e900ca
:1072a0000080400090407800114798001e4178000f
:1072b0000280fb000000e800ee009000008040002b
:1072c000904078001e40900080cf500008003a00a7
:1072d0009e4178000380fb000080e800ee009000f3
:1072e00000804000104078001e4f400060023700d0
:1072f0001e427800634f42005d0237001e4fe800d7
:107300009e4078000180fb00ee009000008040006d
:10731000104078007c0207001e4fe800540237003e
:107320001e4fe8001e4178000280fb00ee00900036
:1073300000804000104078008d0207001e4fe800da
:107340004b0237008e4890000040eb0080cf500089
:107350000f0032002e4090000040e90020479800c6
:10736000ae4090000040eb0080cf500005003a0096
:107370000040eb00004f98009e41780063cf410031
:107380003b0237003e429000044f7800380237003d
:1073900010c0b300004f98009e4078000180fb00b1
:1073a0000000e800ee0090000080400010407800ef
:1073b0009e40780000c05000304798001e41780081
:1073c0000280fb000080e800ee009000008040009a
:1073d00090417800234798003e429000044f780087
:1073e000230237001e4fe8009e4078000180fb001a
:1073f000ee0090000080400010407800d7efb7000a
:107400001e4fe8001a0237001e4fe8001e417800a8
:107410000280fb00ee0090000080400010407800e9
:107420000080fb00030307001e4fe8001002370036
:107430001e4fe8009e4178000380fb00ee009000a4
:1074400000804000104078000080fb00f902070037
:10745000150307001e4fe800050237001e4fe80025
:107460001e4278000480fb00ee0090000080400087
:10747000104078000084fb00270307000080fb0019
:1074800088007800540207001e4fe800f80137001a
:107490001e4fe8009e4078000180fb00ee00900047
:1074a00000804000104078008080fb001e41780082
:1074b0000280fb000000e8006e0190000000410027
:1074c000104078000080fb00430207001ecfe80058
:1074d000e701370080002000d60207001e4fe800b9
:1074e000e301370080002000d2020700ee0207000f
:1074f0001e4fe800de013700070307000080fb0095
:1075000081002000340207001e4fe800d801370038
:107510001e4fe8009e4178000380fb00ee009000c3
:1075200000804000104078000080fb0081002000b7
:10753000290207001e4fe800cd0137001e4fe8006a
:107540001e4278000480fb00ee00900000804000a6
:1075500010407800d6efb700d6cfbf00b6080700be
:107560001e4fe800c2013700cd42a900cd62a9003c
:107570001e4fe800be013700cd42a800cd62a80032
:107580001e4fe800ba013700e4c2a9001e4fe80010
:10759000b7013700e4c2a8001e4fe800b40137006d
:1075a000e2f0a9000000eb00800c8800cca2a9004a
:1075b0001e4fe800ae01370070402000800c8800ac
:1075c000e2f0a800801a260001002000e7ea070088
:1075d0001e4fe800a6013700e4a2a9001e4fe800f4
:1075e000a3013700e4a2a8001e4fe800a001370065
:1075f000e4e2a8001e4fe8009d013700e4e2a90084
:107600001e4fe8009a013700e462a8001e4fe80010
:1076100097013700e462a9001e4fe800940137008b
:107620001e4fe8008040eb000040eb00050407001f
:107630008f0137001e4fe80011c0b3000040eb007f
:10764000000407008a0137001e4fe80011c0b30094
:1076500010c0b300fb030700850137001e4fe80090
:10766000bf030700820137001e4fe800aa0207008f
:1076700000457800a802070080447800a6020700b1
:1076800000447800a40207008a417800094178008c
:107690008840780088030700750137001e4fe80016
:1076a0009e4078000180fb00ee00900000804000ca
:1076b000904178001e4178000280fb000000e80045
:1076c000ee00900000804000104178001e427800db
:1076d0000480fb000080e800ee0090000080400085
:1076e000904078001e4278000480fb006300400058
:1076f0006e02900000004200104078006e03070008
:107700001e407800644f4000590137001e4fe800ca
:107710009e4078000180fb00ee0090000080400059
:10772000904178001e4178000280fb000000e800d4
:10773000ee00900000804000104178001e4278006a
:107740000480fb000080e800ee0090000080400014
:10775000904078001e4278000480fb0063004000e7
:107760006e029000000042001040780014c0b30088
:10777000d60207001e407800644f40003c013700ed
:107780001e4fe8009e4078000180fb00ee00900054
:107790000080400010407800ac0207001e4fe80057
:1077a000330137001e4fe8001e4178000280fb00c5
:1077b000ee00900000804000104078001f04070099
:1077c0001e4fe8002a0137001e4fe8009e41780056
:1077d0000380fb000000e800ee0090000080400005
:1077e000904078001e4278000480fb006e019000fb
:1077f0000000410010407800c80307001ecfe800d9
:107800001b0137001e4fe8009e4078000180fb00fe
:107810000080e800ee0090000080400010417800f9
:107820009e4178000380fb000000e800ee0090001d
:1078300000804000904078001e4278000480fb00e9
:10784000ee0190000080410010407800ff08070022
:107850001e407800634f4000050137001e4fe800ce
:107860009e4078000180fb000000e800ee009000e0
:1078700000804000904078001e4178000280fb00ac
:107880006e01900000004100104078000041eb00c4
:10789000ee0807001ecfe800f50037001e4fe80095
:1078a0001d02070046080700ff010700f00037002f
:1078b0001e4fe8009e4178000380fb00ee00900020
:1078c00000804000104078003d080700f6010700e6
:1078d0001e4fe800e60037000040eb0038080700c4
:1078e000f10107001e4fe800e10037001e4fe800dd
:1078f0000902070032080700dd0037001e4fe800cc
:107900001e4278000480fb00ee00900000804000e2
:10791000104078002a0807001e4fe800d400370006
:10792000f0c0b30086080700df0107001e4fe80023
:10793000cf0037000040eb0081080700da010700a4
:107940001e4fe800ca0037001e4fe800f201070092
:107950005c080700c60037001e4fe8009e40780014
:107960000180fb00ee009000008040001040780095
:10797000540807001e4fe800bd0037003e0807000e
:107980001e4fe800ba003700280807001e4fe80025
:10799000b7003700fe070700c30107001e4fe800cd
:1079a000b30037001e4fe8001e4178000280fb0044
:1079b000ee0090000080400010407800d8efb70043
:1079c000d8cfbf00d90707001e4fe800a800370036
:1079d0001e4fe8009e4178000380fb00ee009000ff
:1079e00000804000104078000084fb00ca010700be
:1079f0000080fb0088007800340107001e4fe8007b
:107a00009b0037001e4fe8001e4278000480fb00f8
:107a1000ee00900000804000104078008080fb0065
:107a20001e4178000280fb000000e8006e0190001b
:107a300000004100104078000080fb002301070097
:107a40001ecfe8008a0037001e4fe8009e417800f4
:107a50000380fb00ee0090000080400010407800a2
:107a6000b10507001e4fe800810037001e4fe800f7
:107a70001e4278000480fb00ee0090000080400071
:107a800090407800114798000a0037001e4fe80028
:107a90001e4178000280fb00ee0090000080400054
:107aa00010407800a00507001e4090000040e9004b
:107ab000104798009e4090000040eb0080cf50009f
:107ac000f2ff3a006a0037001e4fe8004100200034
:107ad0000000eb00c00007009e4178000380fb001f
:107ae000ee00900000804000104078000080fb0015
:107af00041002000b8000700870107000080fb005c
:107b000081002000b4000700810020000000eb008d
:107b1000b10007004100200020002000ae00070057
:107b20001e4fe800520037001e4fe80041002000c1
:107b30000000eb00a80007001e4278000480fb0054
:107b4000ee00900000804000104078000080fb00b4
:107b500041002000a00007006f0107000080fb002b
:107b6000810020009c0007006b0107000080fb00e3
:107b70008100200098000700410020002000200024
:107b8000950007001e4fe800390037001e4fe8003f
:107b90006101070088000700350037001e4fe8002c
:107ba0009e4078000180fb00ee00900000804000c5
:107bb000104078001e4fe8007f0007002c003700bf
:107bc0001e4fe8008000070037010700280037003b
:107bd0001e4fe8001e4178000280fb00ee0090007e
:107be00000804000104078008080fb0000f0200002
:107bf00000804000500798005e0090001040780020
:107c0000290107001e4fe800190037001e4fe80049
:107c10009e4178000380fb00ee0090000080400051
:107c2000104078008080fb0000f0200000804000c1
:107c3000500798001e4fe8001e4278000480fb00a9
:107c4000ee0090000080400010407800de009000c0
:107c5000804878001e4fe800050037001e4fe800fe
:107c600003003700000000000100370000000000a2
:107c7000e1cfbf008080fb00e00f2000808060002b
:107c80000000eb00808f500004003a006e48900026
:107c90009e40780080cf500055fc39004f05780099
:107ca0004f04be000080fa00000006000000fa0049
:107cb0000040eb00e2efb7000040eb00e3efb7005d
:107cc0000000eb00207f88000080fa000000060022
:107cd0000000fa00e7eb070020878800e0eb0700d0
:107ce000408788004087800030878800400e210050
:107cf0008040eb0062002000030020007bee0700c4
:107d00000080fa00000006000200fa00004f780030
:107d10001e4078000080fb0001002000520d200072
:107d20000289b900020178006002b900840178007c
:107d300003014100530d20000300b8000101410080
:107d400082007800a200200003002000cee6070099
:107d50000001be00100020000100200002004000d1
:107d60008380480001e907000080fa000000060057
:107d70000200fa00004f78001e4078000080fb00ef
:107d800001002000425521000289b900020178005b
:107d90006002b900840178000301410043552100cd
:107da0000300b8000101410082007800efe80700fd
:107db0000080fa00000006000200fa00004f780080
:107dc0000080fa00000006000000fa00becfbf00ed
:107dd0000080fa00000006000a00fa003007980050
:107de00041079800100280004500de0067406000f7
:107df0000080fb002007980090028000000f7800b0
:107e0000ff3ffc0011028000f0f12f008080600035
:107e1000000c200000807000100288001e00780016
:107e20009002880000008800e07f80008000eb0066
:107e30000108780071fd20009140780010c0b30067
:107e400080cf500006003600d7cfbf000080fb0077
:107e50000000e9006600b90000007800010037006a
:107e60000000eb0000017800ce0090003e00900082
:107e70009d090700e07f80003100200001087800a4
:107e80009002800010079800ff3ffc002e00900039
:107e900000407800674060000080fb0067006000e1
:107ea0004500dd0012028000f1f12f008100610029
:107eb00000807000100288001e0090009002880070
:107ec000000088000080fa00000006000a00fa00a6
:107ed0003007980041079800100280004500de003e
:107ee000674060000080fb0020079800900280003f
:107ef000000f7800ff3ffc0011028000f0f12f001e
:107f000080806000000c200000807000100288005b
:107f10001e0078009002880000008800e07f80004a
:107f20008000eb000108780071fd2000914078008e
:107f300010c0b30080cf500006003600d7cfbf007e
:107f40000080fb000000e9006900b9000000780033
:107f5000010037000000eb0000017800ce00900027
:107f60003e0090006f090700e07f80003100200094
:107f7000010878009002800010079800ff3ffc0085
:107f80002e00900000407800674060000080fb00f9
:107f9000670060004500dd0012028000f1f12f0053
:107fa0008100610000807000100288001e009000b7
:107fb00090028800000088000080fa00000006009f
:107fc0000200fa00000f7800e422a90071fd2000f1
:107fd0009140780010c0b30080cf500006003600fa
:107fe000d7cfbf000080fb000000e9006600b900a9
:107ff00000007800010037000000eb0080007800ee
:108000001e00780056090700beefb700d6cfbf00ac
:108010000080fb00e20060000000eb00808f500059
:1080200001003a00e422a800becfbf000080fa00a1
:10803000000006000200fa00000f7800e422a90008
:1080400071fd20009140780010c0b30080cf500037
:1080500006003600d7cfbf000080fb000000e9001b
:108060006600b90000007800010037000000eb0056
:10807000800078001e0078004a090700beefb700b4
:10808000d6cfbf000080fb00e20060000000eb00e4
:10809000808f500001003a00e422a800becfbf004c
:1080a0000080fa00000006000200fa00004f78008d
:1080b000207f80008000e80000082000808f5000b2
:1080c00002003600e16fa80011003700527f8000e7
:1080d000e2cfbf008080fb00810041009e48780015
:1080e0000040e800e2efb700e2cfbf008040780038
:1080f0000040eb0080cf500002003d000040eb004c
:10810000e2efb700207f80000000e800207f8800b9
:108110000080fa00000006000200fa00f17e8000f4
:108120000000eb00808f500003003a00e18fa800b0
:108130000040eb0010003700417f8000e07e8000af
:1081400080804000114f78000000e800e07e880049
:10815000f07e80000000e900f07e8800e17e800073
:10816000f00f2000808f5000020036000000eb006e
:10817000e07e88001e4078000080fa0000000600c3
:108180000200fa00207f8000104798009e40900077
:10819000f0c3b30080cf500002003600f0c3b3003c
:1081a00010479800907f80009e4090000148780022
:1081b00010c0b300004f780014003700917f80009a
:1081c0001e4178000280fb0000814000537f800048
:1081d000e3cfbf008080fb008180410091407800a8
:1081e000014978000040e800e3efb700e3cfbf00ab
:1081f000804078000040eb0080cf500002003d003e
:108200000040eb00e3efb7001e4fe8001e40900077
:108210009e40780080cf5000e8ff3600217f80002c
:108220001e4090000080fb0000805000207f8800ee
:10823000907f80008040eb000204200003002000bb
:108240002aed07000080fa00000006000400fa0092
:10825000204798000040eb00004f780011c0b300a9
:1082600030c0b3002d010700c0cfbf0080407800b0
:108270000040eb0080cf500002003d0010c0b30072
:10828000004f780002c8b300ae40900080c0b30039
:108290003f010700c0cfbf000080fb00000040008e
:1082a000804078001e40780000c07000004f7800c9
:1082b0001e4078007cff070011c0b30020c0b3004f
:1082c000160107000080fa00000006000800fa000e
:1082d000204798003147980042479800534798003c
:1082e000644798000040eb00004f78000040eb002e
:1082f0001047980011c0b30030c0b3000701070059
:10830000c0cfbf00804078000040eb0080cf50001d
:1083100002003d0010c0b300004f78000041eb00a8
:10832000de40900080c0b30019010700c0cfbf003d
:108330000080fb0000004000804078001e40780074
:1083400000c07000004f7800ee4090000040eb004d
:1083500080cf5000020032001e40780052ff07001c
:108360000040eb00004f7800c0cfbf008040780095
:108370000040eb0080cf500002003d0010c0b30071
:10838000004f78000041eb00ce40900080c0b30069
:10839000ff000700c0cfbf000080fb0000004000ce
:1083a000804078001e40780000c07000004f7800c8
:1083b000ee4090000040eb0080cf50000200320001
:1083c0001e40780038ff07000040eb00004f7800a7
:1083d000c0cfbf00804078000040eb0080cf50004d
:1083e00002003d0010c0b300004f78000041eb00d8
:1083f000be40900080c0b300e5000700c0cfbf00c2
:108400000080fb0000004000804078001e407800a3
:1084100000c07000004f7800ee4090000040eb007c
:1084200080cf5000020032001e4078001eff07007f
:108430001e407800104798000040eb00004f780085
:10844000c0cfbf00804078000040eb0080cf5000dc
:1084500002003d0010c0b300004f780002c8b30016
:10846000ae40900080c0b300c9000700c0cfbf007d
:108470000080fb0000004000804078001e40780033
:1084800000c07000004f7800ee4090000040eb000c
:1084900080cf5000020032001e40780002ff07002b
:1084a00011c0b30020c0b3009c0007001e40900024
:1084b0000080fa00000006000400fa00004f780077
:1084c00011479800224798003347980011c0b30025
:1084d00030c0b30091000700c0cfbf0080407800db
:1084e0000040eb0080cf500005003500f1c1b30023
:1084f00050c0b30089000700e14fa8001600370004
:108500008040eb0010c0b300840007000041eb0086
:10851000be40900080c0b3009d0007000041eb000a
:10852000ae40900080c0b300990007000041eb000e
:108530009e40900080c0b3009500070002c8b300c1
:108540009e40780080c0b3009100070011c0b300c6
:1085500020c0b300710007000080fa000000060090
:108560000400fa00889fbe008a1f780000e2240001
:10857000000f7800a0c0b300b00007000042eb007d
:108580008041eb0002cdb30041c0b3000040eb00de
:108590004eff0700204798002e4090000080fb000f
:1085a000e40060000000eb00808f500005003a00fe
:1085b0001e0fe9009e0078000000eb00808f500045
:1085c000eeff3a009e0078000000eb00808f500024
:1085d00002003a00e14fa8001600370090c0b30037
:1085e00096000700ccfe070000457800cafe070091
:1085f00080447800c8fe070000447800c6fe0700eb
:108600000042eb008a4178000941780088407800f8
:108610002eff0700a0c0b300880007000042eb0057
:108620008041eb0002ccb3008040eb000040eb0047
:1086300026ff07004f0578004f04be000080fa00b7
:10864000000006000600fa004047980051479800d5
:1086500000e22400000f7800a0c0b30077000700fc
:108660000042eb008041eb0002cdb30041c0b300fb
:108670000040eb0015ff0700204798002e409000b7
:108680000080fb00e40060000000eb00808f5000e1
:1086900005003a001e0fe9009e0078000000eb0084
:1086a000808f5000eeff3a009e0078000000eb0043
:1086b000808f500002003a00e14fa80015003700fb
:1086c00090c0b3005d0007004e409000004278006b
:1086d0008041eb000041eb008040eb000040eb00ec
:1086e000fafe0700de4090000040eb0080cf500013
:1086f00008003200a0c0b300500007000042eb00a9
:108700008041eb0002ccb3008040eb000040eb0066
:10871000eefe07000080fa00000006000400fa00e8
:108720002047980031479800ae4090000040eb0091
:1087300080cf5000130032000040eb00beefb700c6
:108740003e409000bfefb7000040eb00004f7800c4
:108750000700370047000700bfcfbf000080fb00c5
:108760000000d10000407800bfefb7001e4fe800c6
:108770002e4090009e40780080cf5000f5ff3900d9
:1087800001003700000000000080fa000000060031
:108790000600fa00204798003147980042479800a9
:1087a000ae4090000040eb0080cf500002003a0045
:1087b0000040eb001f0037003e409000beefb700c6
:1087c0004e409000bfefb7000040eb00c0efb70095
:1087d0000040eb00004f780011003700c0cfbf0011
:1087e0000080fb000000d10000407800c0efb7001f
:1087f00020000700becfbf000080fb000000d100ba
:1088000000407800beefb700bfcfbf000080fb0084
:108810000000d10000407800bfefb7001e4fe80015
:108820002e4090009e40780080cf5000ebff390032
:10883000c0cfbf000080fa00000006000200fa006e
:10884000004f780031c0b30040c0b300b3ff070051
:1088500002c1b3009e40780050c0b300ccff0700b7
:1088600011c0b30020c0b300acff07000080fa00c5
:10887000000006000000fa00da42a800dc82a9002d
:10888000becfbf000080fb00610060008040780028
:108890000040eb0080cf500001003200dc82a800d5
:1088a000e422a80000000000da42a900bfcfbf0008
:1088b0000080fb00e10060000000eb00808f5000b2
:1088c00001003a00dc82a90000000000da42a800a2
:1088d000bfcfbf000080fb006100600080407800d7
:1088e0000040eb0080cf500001003200dc82a80085
:1088f000c0cfbf000074a100c0efb700da42a900ea
:10890000da42a800e422a900da42a900000000002f
:10891000da42a80000000000d0168000e8006000e5
:108920000000eb00808f50000500320001fc2000a9
:108930009140780000c8b30000c07000c0efb700dd
:10894000da42a9000080fa00000006000000fa00e8
:1089500001fe20009140780000cfb30000c060000d
:10896000e0efb70011178000000220008080600057
:108970000000eb00808f500001003200e06fa80083
:108980001117800000042000808060000000eb00d0
:10899000808f500001003200e04fa80010178000c7
:1089a000e80060000000eb00808f500001003a00fa
:1089b000e02fa800111780000008200080806000d0
:1089c0000000eb00808f500001003a00e00fa8008b
:1089d000a10e2100914078000040eb0080cf5000b4
:1089e00001003200e0cfa8000040eb00eaf0b70041
:1089f000917f8000e0cfbf0080487800907f8000aa
:108a00008000e800e1cfbf008048780001fe200030
:108a100091407800f0c8b30000c06000e0efb700fc
:108a20000040eb00e1efb700cd42a900cd62a90004
:108a3000907f80008040eb000204200003002000b3
:108a40002aeb07000080fa00000006000200fa008e
:108a50000040eb00004f780008003700317f8000b5
:108a60001e4178000280fb004200dd008080400053
:108a70000040eb00804878001e4fe8009e407800e0
:108a8000f0c1b30080cf5000f4ff36000080fa0040
:108a9000000006000a00fa0040079800817f80006d
:108aa0004e009000100078000000e80000804000b8
:108ab000104078000080fb0020079800ae00900076
:108ac000d0032000808f500002003400e1cfa800c6
:108ad000b3003700817f80004e00900010007800c6
:108ae00000804000104078000080fb0030079800b4
:108af0000000eb00100798000000eb00000f78006a
:108b00000a003700317f80001e0078004200dd003f
:108b100000804000104078000080fb009e00900024
:108b200000804000100798001e0fe8009e007800ab
:108b3000f0012000808f5000f2ff3400317f800070
:108b40003e0090004200dd000080400010407800b0
:108b50000080fb009e0090000080500010079800ed
:108b6000013020001e009000808050002e009000f8
:108b7000808f500002003d00e1cfa8008800370040
:108b8000be009000f0012000808f500002003400f1
:108b9000e1cfa80082003700317f80003e009000c6
:108ba0004200dd0000804000904078000040eb0073
:108bb00080cf500049003200317f80003e0090009d
:108bc0004200dd0000804000104078000080fb0083
:108bd000f12f20000080500020079800317f800096
:108be0003e0090004200dd000080400090009000b8
:108bf000010f780010003700717f80001e007800a0
:108c000080804000727f8000337f80003e009000b3
:108c10004200dd0000804100104078008081fb00b0
:108c20001e007800008041000000410010407800e4
:108c3000804878001e0fe8002e0090009e0078000b
:108c4000808f5000ecff35000000eb00000f780033
:108c50001e003700317f80001e0078004200dd00da
:108c60000080400090009000327f80003e00900025
:108c70004200dd000000410010009000808f500095
:108c800011003400317f80001e0078004200dd00ba
:108c900080804000327f80001e0078004200dd00ae
:108ca0000000410010019000337f80003e009000e2
:108cb0004200dd0000804100104078000080fb0091
:108cc00000005100900098001e0fe8009e00780000
:108cd000f0012000808f5000deff3400317f8000e3
:108ce0003e0090004200dd0080804000827f8000d6
:108cf0004e009000100078000000e80000004100e5
:108d00001040780080487800317f80003e0090005d
:108d10004200dd00008040009e009000110098009d
:108d20004e009000100078008080e8004e00900017
:108d3000010878000000eb00000f78000f003700fa
:108d4000717f80001e0190001e007800000041002d
:108d500000814000807f8000ce009000910078006c
:108d60000100400010407800004978008100e800d0
:108d70004e009000010878001e0fe800317f80004f
:108d80003e0090004200dd0000804000104078006e
:108d90008080fb001e007800808f5000e8ff3c00c0
:108da0000080fa00000006000200fa00004f780080
:108db000114798009e407800f0c1b30080cf50006a
:108dc00009003e00317f80001e4178000280fb00d8
:108dd0004200dd0000804000904078000040eb0041
:108de00080cf500002003a00e1afa8001800370021
:108df000317f80001e4278000480fb004200dd00cd
:108e00000080400010407800727f8000337f800037
:108e10001e4278008480fb00c208dd008180410092
:108e2000910090000101410080407800020078002c
:108e3000d2f707001e4090000040e900104798005c
:108e40009e4090000040eb0080cf5000e8ff3a00c9
:108e50000080fa00000006000600fa000000eb00a7
:108e6000000f78000000eb00100798000000eb00f6
:108e7000200798000000eb00200798000a00370048
:108e8000317f80002e0090004200dd000080400015
:108e9000104078000080fb001e0f40002e00900064
:108ea0000000e80020079800ae009000f0012000cc
:108eb000808f5000f2ff34000000eb002007980084
:108ec0000b003700717f80002e0090000080400072
:108ed000104078000080fb009e0090000080400061
:108ee000100798002e0090000000e800200798006e
:108ef000ae0090001e007800808f5000f1ff35001a
:108f0000917f80001e007800004078008048780043
:108f1000907f80008000e8001e0078004880de001e
:108f20000040780080487800907f80008080e800d2
:108f30001e0090000040780080487800907f8000fc
:108f4000e30040001e0090004880de0000407800f2
:108f500080487800907f80008040eb000204200071
:108f600003002000e1e907000080fa00000006008d
:108f70000000fa000000eb00d07e88000000eb004b
:108f8000e07e88000000eb00f07e88000080fa00a0
:108f9000000006000600fa0020079800807f80008d
:108fa000ae00900091007800010040001040780071
:108fb0000080fb00100798008100e8002e00900060
:108fc00001087800f17e80001e0090008080400043
:108fd00000102000808f500002003600e1efa80052
:108fe0001f0037000000eb00000f7800180037006a
:108ff000407f8000d27e800082014000807f800020
:10900000ae00900091007800010040001040780010
:10901000804978000200e800d07e88008100e800e6
:109020002e00900001087800d17e8000f00f200013
:10903000808f5000020036000000eb00d07e8800d8
:10904000f07e80000000e800f07e88001e0fe8003f
:109050001e0090009e007800808f5000e4ff3900d1
:109060000080fa00000006000200fa00207f800065
:10907000104798009e40900000c4b30080cf50007d
:109080000200360000c4b300104798000040eb0017
:10909000004f780014003700917f80001e41780057
:1090a0000280fb0000814000537f8000e3cfbf00bf
:1090b0008080fb0081804100914078000149780068
:1090c0000040e800e3efb700e3cfbf008040780046
:1090d0000040eb0080cf500002003d000040eb005c
:1090e000e3efb7001e4fe8001e4090009e4078005e
:1090f00080cf5000e8ff3900217f80001e409000a3
:109100000080fb0000805000207f8800907f80005e
:109110008040eb00020420000300200073e90700f8
:109120000080fa00000006000200fa00004f7800fc
:10913000417f8000d07e8000808040009e48780083
:109140000000e800d07e8800d17e8000f00f200073
:10915000808f5000020036000000eb00d07e8800b7
:10916000f07e80000000e800f07e88000080fa00b9
:10917000000006000400fa00204798000000eb0001
:10918000000f78002e4090000080fb00e40060009b
:109190000000eb00808f5000010032001e30a00064
:1091a0002e4090000080fb00e80060000000eb0013
:1091b000808f5000010032001e20a0002e40900041
:1091c0000080fb00f00060000000eb00808f50008a
:1091d00002003200000820001e0f70001e00780000
:1091e0000080fa00000006000400fa002047980002
:1091f0000000eb00000f78002e4090000080fb0084
:10920000e80060000000eb00808f50000100320099
:109210001e20a0002e4090000080fb00e4006000b3
:109220000000eb00808f5000010032001e30a000d3
:10923000ae4090000040eb0080cf500001003d00a8
:109240001e40a0001e007800004078000080fa0058
:10925000000006000400fa00204798002e4090000d
:10926000410020000100dd00004f78002e409000fa
:109270000080fb004400de00104798001e40900074
:109280001e4070000080fa00000006001200fa0084
:10929000100280004500de00674060000080fb0097
:1092a000000f98009002800020079800ff3ffc000c
:1092b00011028000f0f12f0080806000000c20007f
:1092c00000807000100288002e009000900288003c
:1092d00000008800e07f80008000eb00010878003b
:1092e000e402a900d842a800e422a900e442a900af
:1092f000e862a800d5fd0700cd42a800cd62a80015
:10930000becfbf009bff0700607e8800c0cfbf00bc
:1093100098ff0700707e8800c2cfbf0095ff07004e
:10932000807e8800c3cfbf000080fb00907e880055
:10933000c5cfbf000080fb00c800dd00c4cfbf0068
:109340000080fb0000804000a07e8800e882a90029
:1093500091fc2000914078000040eb0080cf50004d
:10936000030032000000eb001007980002003700f5
:10937000807e800010079800cacfbf000080fb00ed
:10938000c800dd00c8cfbf000080fb0000804000a7
:1093900030079800be0090001e009000f403070004
:1093a000907e88000000eb00000f78001d00370061
:1093b000000024001e00400090407800014f9800fb
:1093c0009e00e800000024000080400090407800eb
:1093d000114f98000e48900083ff07007c4060000a
:1093e000004f98001e4890007fff07007c406000ff
:1093f000104f98001e48900096ff0700104f9800ed
:109400001e0078000001d1009e4890000e48900098
:1094100000c07000010024008100410080487800f5
:109420001e8fe800f03f20009e007800808f5000e3
:10943000dfff36000000eb00000f7800150037005a
:10944000000024001e00400090407800214f98004a
:10945000f01f20009e00500000002400008040000b
:1094600090407800314f9800000024001e0040001a
:10947000be48900001487800f01f20009e00500078
:109480000000240000804000ae48900001487800b1
:109490001e0fe800f00f20009e007800808f500023
:1094a000e7ff3600917e80000080eb00808f500047
:1094b0001a003200917e800000002c0000804000e5
:1094c000907e8800907e80006100600060079800b8
:1094d000907e80000000d100907e8800907e800009
:1094e000f11f200000805000907e8800917e800057
:1094f0000000240000804000907e8800ee00900074
:109500000000eb00808f500004003200917e80004c
:109510000000280000807000907e880020fd200060
:1095200010407800beefb70020fd20000000e800ea
:1095300010407800bfefb700cd42a900cd62a9006e
:10954000e07f800031002000010878009002800058
:1095500070079800ff3ffc000e0890000040780064
:10956000674060000080fb00670060004500dd0090
:1095700012028000f1f12f00810061000080700074
:10958000100288007e009000900288000000880091
:10959000917f8000becfbf0080487800907f800020
:1095a0008000e800bfcfbf0080487800907f800037
:1095b0008040eb0002042000030020004be807007d
:1095c0000080fa00000006000600fa0040479800fc
:1095d000514798004e4090008080fb005e40900014
:1095e0000080fb004800dd0000804000100798006c
:1095f0000040eb00004f7800070037001e0090008d
:10960000104078009e0090008100e800110798004b
:10961000a5fa07001e4fe8009e4078000040eb00ce
:1096200080cf5000f5ff3d000080fa0000000600ea
:109630002800fa0030179800817f80003e109000cb
:109640001000780080804000114178004247980067
:109650008000e8003e10900001087800807f8000c4
:10966000be1090009100780001004000104078008a
:109670000080fb00100798008100e8003e10900079
:10968000010878009e00900000022000808f5000aa
:109690000200360000022000100798009e00900093
:1096a0000000eb00808f50001f003200ce40900081
:1096b00000cfb30080cf500007003a00650047009c
:1096c0000402200005002000000178006001200055
:1096d00001002000f1f107000000eb00000f78000e
:1096e00007003700907f80009e0040006500470023
:1096f0001e00400010407800804878001e0fe800ef
:109700001e0090009e007800808f5000f5ff390009
:10971000907f80008040eb000204200003002000c6
:10972000f2e7070001003700000000000080fa00a7
:10973000000006002600fa0020179800817f8000b4
:109740002e109000100078008080400011417800b9
:10975000224798008000e8002e1090000108780051
:10976000817f80002e1090001000780080804000e3
:1097700011417800124798008000e8002e109000f8
:10978000010878009e40900000c2b30080cf5000d6
:109790000200360000c2b300104798009e409000bf
:1097a0000040eb0080cf5000200032000040eb0072
:1097b000004f78000d0037001e4078000081fb004c
:1097c000807f8000ae109000910078000100400082
:1097d00010407800e3014700807179008100e800c3
:1097e0002e109000010878001e4fe8001e409000e7
:1097f0009e40780080cf5000efff3900ae409000cf
:1098000000cfb30080cf500009003a00630047004a
:109810000402200005002000000178006001200003
:1098200001002000ecf107000100370000000000fb
:109830000080fa00000006000200fa00004f7800e5
:109840009e4078000180fb00e40060000000eb0017
:10985000808f500002003200da42a8000100370079
:10986000da42a9009e4078000180fb00e800600019
:109870000000eb00808f500002003200dc82a80064
:1098800001003700dc82a9009e4078000180fb00c7
:1098900061006000804078000040eb0080cf500005
:1098a00003003200e402a900d842a80002003700f9
:1098b000e402a800d842a9009e4078000180fb0085
:1098c000e20060000000eb00808f500002003200d8
:1098d000e422a90001003700e422a8000080fa0079
:1098e000000006000200fa000040eb00004f780084
:1098f000d0168000e80060000000eb00808f500070
:10990000010032001e14a000d0168000e4006000a8
:109910000000eb00808f5000010032001e04a00008
:109920001e4078000080fa00000006000200fa00e5
:10993000004f78009e4078000180fb00e20060004c
:109940000000eb00808f500002003200ec62a800a3
:1099500001003700ec62a9009e4078000180fb0006
:1099600061006000804078000040eb0080cf500034
:1099700003003200e442a900e862a80002003700b8
:10998000e442a800e862a9000080fa000000060096
:109990000200fa000040eb00004f780050178000f2
:1099a000e80060000000eb00808f500001003200f2
:1099b0001e04a0001e4078000080fa00000006008f
:1099c0000400fa002047980080002000000f780073
:1099d00071fd20009140780010c0b30080cf50008e
:1099e00005003e009e0078002e4090000203070014
:1099f000beefb7000a003700d7cfbf000080fb00e2
:109a00000000e9006700b90000007800000178005c
:109a10009e0078002e40900009030700beefb700bb
:109a2000becfbf000080fa00000006000000fa0070
:109a3000da42a800d00420000100200088050700b9
:109a4000ec62a900e442a800e862a900d00420006a
:109a50000100200082050700da42a900d00420009e
:109a6000010020007e050700e442a900e862a8008a
:109a70000080fa00000006000000fa00da42a900a7
:109a8000d00420000100200075050700ec62a90049
:109a9000e442a800e862a900d004200001002000f0
:109aa0006f050700da42a800d00420000100200062
:109ab0006b050700e442a900e862a8000080fa00f4
:109ac000000006000400fa002047980080002000f3
:109ad000000f7800ec62a90071fd20009140780031
:109ae00010c0b30080cf50000a003e009e007800f6
:109af0002e409000e8020700f1fb20009140780022
:109b00000040eb0080cf50000b003200e14fa80076
:109b1000090037009e0078002e409000fc020700ec
:109b2000f1fb2000914078000040eb0080cf500016
:109b300001003200e14fa8000080fa00000006009a
:109b40000c00fa00204f98000040eb00004f780016
:109b50008000200010079800100280004500de0001
:109b6000674060000080fb00400798009002800082
:109b700020079800ff3ffc0011028000f0f12f0049
:109b800080806000000c20000080700010028800bf
:109b90002e0090009002880000008800e07f800086
:109ba0008000eb000108780071fd200091407800f2
:109bb00010c0b30080cf500006003e002e49900038
:109bc0009e0090001e407800ef020700beefb70035
:109bd000050037002e4990009e0090001e4078003e
:109be00004030700beefb700e442a900e862a80042
:109bf000e07f8000310020000108780090028000a2
:109c000030079800ff3ffc004e00900000407800b5
:109c1000674060000080fb00670060004500dd00d9
:109c200012028000f1f12f008100610000807000bd
:109c3000100288003e00900090028800000088001a
:109c4000becfbf000080fa00000006000e00fa0040
:109c5000204f9800314f9800424f98000040eb0091
:109c6000004f7800100280004500de006740600071
:109c70000080fb00400798009002800020079800b9
:109c8000ff3ffc0011028000f0f12f008080600097
:109c9000000c200000807000100288002e00900050
:109ca0009002880000008800e07f80008000eb00c8
:109cb0000108780071fd20009140780010c0b300c9
:109cc00080cf500005003600d0132000d008880057
:109cd00080ccb3002047980004003700d004200057
:109ce000d008880080c2b30020479800ec62a8002a
:109cf000e442a800e862a90000142000010020004e
:109d0000d70407003e48900000c0e800304f98009c
:109d10000000eb00f008880050c5b300beefb700ac
:109d2000ec62a900000a200001002000cc0407001a
:109d30000000eb00a00888008760a9001fe1a800d0
:109d40003e4890000040e900304f98000040eb0092
:109d5000104798002800370060178000704fb2004d
:109d6000beefae008040b3008760ae00feff37005c
:109d700060178800e442a800e862a9008760a90093
:109d8000becfbf0000404000beefb70060178000ac
:109d900000407800bfefb700be4890000040eb00e5
:109da00080cf500008003a00ce4890000040eb0001
:109db00080cf500004003a00bfcfbf000034a000a5
:109dc000bfefb70005003700f1fb2000914078009d
:109dd00070cfb30000c06000bfefb7008760ae0077
:109de000feff3700ec62aa008760a9001e409000c9
:109df0000040e800104798009e40900070c0b300fb
:109e000080cf5000d4ff3400bfcfbf008760ae00ca
:109e1000feff3700601788008760a9009e40780029
:109e20000040eb0080cf500007003200be48900099
:109e30000040eb0080cf500003003200b6f807006e
:109e4000beefb700020037002e489000beefb7000b
:109e50008760ae00feff3700ec62aa008760a900b1
:109e60008760ae00feff3700e442a900e862a80068
:109e70008760a9002e4090000080fb0001002000b8
:109e8000770407009e4078000040eb0080cf500030
:109e90000a00320050178000e80060000000eb006c
:109ea000808f500005003200e14fa8000040eb0019
:109eb000304f98000040eb00404f98008760ae00a4
:109ec000feff3700000000008760a9002e409000d0
:109ed0000080fb0001002000610407009e40780024
:109ee0000040eb0080cf50000a0032005017800085
:109ef000e80060000000eb00808f500005003a0091
:109f0000e14fa8000040eb00304f98000040eb000c
:109f1000404f980010c0b300004f7800be4890003a
:109f20000040eb0080cf500085ff3a007c003700f6
:109f30000040eb00beefb7000040eb001047980078
:109f40003b0037008760ae00feff37008760a90046
:109f50006017800000407800bfefb700ce48900047
:109f60000040eb0080cf500004003a00bfcfbf009c
:109f70000034a000bfefb70005003700f1fb200060
:109f80009140780070cfb30000c06000bfefb70011
:109f90002e4090000080fb000000e900cf80de0032
:109fa0002f04070050178000e80060000000eb005d
:109fb000808f500006003a008760af000200370033
:109fc000ea62ae00fcff37001421ef000500370005
:109fd0008760af0002003700ea62af00fcff370085
:109fe0001421ef008760a9002e4090000080fb0044
:109ff000010020001a040700becfbf00004040004f
:10a00000beefb70050178000e80060000000eb00d2
:10a01000808f500003003200becfbf000040e80038
:10a02000beefb7001e4090000040e80010479800c7
:10a030009e40900070c0b30080cf5000c1ff34003c
:10a04000bfcfbf008760ae00feff370060178800fb
:10a05000e442a800e862a9008760a90000000000af
:10a0600000000000becfbf000ff807008760ae0001
:10a07000feff3700ec62aa008760a9008760ae008f
:10a08000feff3700e442a900e862a8008760a9004b
:10a090002e4090000080fb0001002000f00307002c
:10a0a0009e4078000040eb0080cf50000800320056
:10a0b00050178000e80060000000eb00808f500027
:10a0c00003003200e14fa8000040eb00404f980031
:10a0d0008760ae00feff3700000000008760a90027
:10a0e0002e4090000080fb0001002000dc030700f0
:10a0f0009e4078000040eb0080cf50000800320006
:10a1000050178000e80060000000eb00808f5000d6
:10a1100003003a00e14fa8000040eb00404f9800d8
:10a120004e4890000080fb000000ea004f00de0077
:10a13000804078004e4890000040e900404f980071
:10a140000040eb0080cf500079ff3a00e442a900c4
:10a15000e862a800e07f800031002000010878005c
:10a160009002800030079800ff3ffc004e009000f6
:10a1700000407800674060000080fb0067006000de
:10a180004500dd0012028000f1f12f008100610026
:10a1900000807000100288003e009000900288004d
:10a1a000000088000080fa00000006000200fa00ab
:10a1b0000000eb00000f780006003700917f800060
:10a1c0001e007800808040000040eb00804878004e
:10a1d0001e0fe8009e007800d0012000808f500004
:10a1e000f6ff3400907f8000fe00400000c5b30001
:10a1f00080487800907f8000ff004000b0c6b30028
:10a2000080487800907f800001022000808040001c
:10a2100030c3b30080487800907f80001102200096
:10a2200080804000f5cfbf0080487800907f80009c
:10a230002102200080804000f6cfbf0080487800d7
:10a24000907f80003102200080804000f7cfbf0067
:10a2500080487800907f80008040eb00020420005e
:10a260000300200021e507000080fa00000006003e
:10a270000000fa00917f800040c2b300804878005f
:10a28000907f80008000e8000040eb00804878006c
:10a29000cd42a900cd62a80010e107008040eb008c
:10a2a000814f500006003200fce00700907f8000e4
:10a2b0008080e80090c9b30080487800040037002f
:10a2c000907f80008080e800a0cab30080487800ba
:10a2d000907f80008040eb000204200003002000fb
:10a2e00002e5070068e5070000242400f1002000d3
:10a2f0009edf07000000fe000080fa00000006005c
:10a300000000fa00917f8000a0c2b300804878006e
:10a31000907f80008000e8000040eb0080487800db
:10a32000eee007008040eb00814f50000500320056
:10a33000907f80008080e80090c9b300804878005a
:10a3400004003700907f80008080e800a0cab3003e
:10a3500080487800907f80008040eb00020420005d
:10a3600003002000e1e407000080fa00000006007e
:10a370000004780081037800060024008a7e8000b3
:10a38000ab7e80000c402000d0168000511780006a
:10a390006c006000c408dd0000807000005b780085
:10a3a00006a0a10007800900000000000c06e900db
:10a3b00004003a0080047800000000000000000063
:10a3c000080037000000000000000000eeff37002a
:10a3d000cb02ae004200370000000000b644780017
:10a3e00006a0a100d0168000511780006c0060000c
:10a3f000c408dd000080700007800900004b780071
:10a40000cc0fb600ce8fb600f1ff3a00090665000a
:10a410000c066c00f1ff3a00d22fed0021003a004b
:10a4200000000000d0168000511780006c00600012
:10a43000c408dd00008070000603e80006a0a1004b
:10a4400086017800005b780006a0a1000780090063
:10a4500000000000000000000000000000000000fc
:10a4600000000000d0168000511780006c006000d2
:10a47000c408dd0000807000005b780006a0a10029
:10a4800007800900000000008b05e90002003a0087
:10a49000030078000000060000000000000000003b
:10a4a000f0ff3700d0168000511780006c0060006c
:10a4b000c408dd0000807000b644780006a0a1004a
:10a4c000005b780006a0a1000780090000000000e2
:10a4d000000000000000000000000000c1ff370085
:10a4e000f0ff2f00000006000000a600dc82a9009b
:10a4f0000000a700dc82a800028009000000000024
:10a50000dc42a8000280090000000000dc42a90033
:10a510000000d1008100e900f3ff3a00dc82a900cd
:10a52000000006000000a600dc82a9000000a700d1
:10a53000dc82a800dc42a8000280090000000000c4
:10a54000dc42a90002800900000000000000d100e8
:10a550008100e900f3ff3a00dc82a9000000060058
:10a560000001eb0068021000da62af000200a000f8
:10a57000dc42a8000000000000000000018009008b
:10a5800000000000dc42a90001800900000000007a
:10a590000241d3000000e900f3ff3a000410de009e
:10a5a000000006000001eb0068021000dc42a80079
:10a5b000000000000000000000000000000000009b
:10a5c0000180090000000000da62af000200a00074
:10a5d000dc42a90001800900000000000241d30014
:10a5e0000000e900f1ff3a000410de000a00090053
:10a5f00000000000000006000070a600ec62a90048
:10a600000070a700ec62a80000000000dc42a80077
:10a610000000000000000000000000000040d20028
:10a620000000a100dc42a900da62af000000a00037
:10a630008100e900f0ff3a00ec62a900000006008a
:10a640000070a600ec62a9000070a700ec62a800f0
:10a650000280090000000000dc42a80000000000a9
:10a660000000000000000000000000000040d200d8
:10a670000000a100da62af000000a0000280090023
:10a6800000000000dc42a9008100e900ecff3a0074
:10a69000ec62a900000006000070a600e862a900b4
:10a6a0000070a600e442a8000070a700e862a800bd
:10a6b0000070a700e442a9000800090000000000a3
:10a6c000dc42a8000b00090000000000dc42a900e9
:10a6d00001000900000000000040d2008100e900f4
:10a6e000edff3a00e862a800e442a9000f0009006b
:10a6f00000000000dc42a800090009000000000082
:10a70000ea62af00bf0fa800dc42a900000006000b
:10a710000070a600e862a9000070a600e442a8004c
:10a720000070a700e862a8000070a700e442a9003a
:10a730002900090000000000dc42a80035000900e3
:10a7400000000000dc42a9002e000900000000000b
:10a750000040d2008100e900edff3a00e862a80065
:10a76000e442a9003000090000000000dc42a8001b
:10a770003300090000000000ea62af00bf0fa8002c
:10a78000dc42a900000006000040d20008000900d9
:10a7900000000000dc42a8000900090000000000e1
:10a7a000ea62af000000a000dc42a9000900090035
:10a7b000000000008100e900f3ff3a00ec62a9000c
:10a7c0000200a600e862a9000200a600e442a80078
:10a7d0000500090000000000dc42a8000b00090091
:10a7e00000000000dc42a900040009000000000095
:10a7f000000006000040d2002a000900000000000e
:10a80000dc42a8003300090000000000ea62af004b
:10a810000000a000dc42a900350009000000000093
:10a820008100e900f3ff3a00ec62a9000200a600f3
:10a83000e862a9000200a600e442a800270009007f
:10a8400000000000dc42a800350009000000000004
:10a85000dc42a90010000900000000000000060012
:020000040000fa
:10a8600012010000000200000000000000080000cb
:10a87000d80400000a90000002000000010200005d
:10a88000030100000902000029000000010100008e
:10a8900000800000fa09000004000000000200002f
:10a8a0000300000000000000092100001101000069
:10a8b00000010000221d00000007000005810000cb
:10a8c0000340000000010000070500000103000034
:10a8d0004000000001000000040300000904000023
:10a8e000340300004d000000690000006300000018
:10a8f000720000006f0000006300000068000000ac
:10a9000069000000700000002000000054000000fa
:10a910006500000063000000680000006e00000099
:10a920006f0000006c0000006f0000006700000076
:10a930007900000020000000490000006e000000c7
:10a94000630000002e000000120300005000000011
:10a9500049000000430000006b0000006900000097
:10a960007400000020000000330000001e030000ff
:10a970004d000000540000004900000030000000bd
:10a980003000000030000000300000003000000007
:10a9900030000000300000003000000030000000f7
:10a9a000000000000000000006000000ff09000099
:10a9b00001a100000119000001290000401500005c
:10a9c00000260000ff000000750800009540000010
:10a9d00081020000190100002940000091020000de
:10a9e000c000000042d400006cd4000070d400000d
:10a9f000a4d40000b6d40000444500004641000045
:10aa0000554c0000545f0000504b00003320000004
:10aa1000000000000001000004140000010000001c
:08aa200001000000000000002d
:020000040000fa
:10aa2800809fbe00821f78000800fa001002800094
:10aa38004500de00674060000080fb00300798009a
:10aa480090028000000f7800ff3ffc001102800098
:10aa5800f0f12f0080806000000c20000080700062
:10aa6800100288001e00780090028800000088000c
:10aa7800e07f80008000eb000108780034c0bf0050
:10aa88000080fb00100798000000200000407800bc
:10aa980034e0b70084e0a900cd22a8001e00900091
:10aaa8000040780034e0b700e07f800031002000eb
:10aab800010878009002800020079800ff3ffc0002
:10aac8003e00900000407800674060000080fb0076
:10aad800670060004500dd0012028000f1f12f00e0
:10aae8008100610000807000100288002e00900034
:10aaf80090028800000088000080fa004f0178006a
:10ab08004f00be00004006003600f800809fbe00df
:10ab1800829fbe00849fbe00869fbe000800fa0088
:10ab2800100280004500de00674060000080fb00e6
:10ab38003007980090028000000f7800ff3ffc006b
:10ab480011028000f0f12f0080806000000c2000ce
:10ab580000807000100288001e00780090028800b3
:10ab680000008800e07f80008000eb00010878008a
:10ab780034c0bf000080fb001007980000002000d0
:10ab88000040780034e0b700b0e607008ec0a900a6
:10ab98009ec0a8001e0090000040780034e0b70076
:10aba800e07f8000310020000108780090028000da
:10abb80020079800ff3ffc003e009000004078000e
:10abc800674060000080fb00670060004500dd0012
:10abd80012028000f1f12f008100610000807000f6
:10abe800100288002e009000900288000000880063
:10abf8000080fa004f03be004f02be004f01be00a6
:10ac08004f00be003600f900004006003600f8008c
:10ac1800809fbe00829fbe00849fbe00869fbe00ac
:10ac28000000fa008780a900b17580000000eb00e1
:10ac3800808f500001003a009780a900a17580001c
:10ac48000000eb00808f500007003200a1758000e3
:10ac580010002000808f500003003200a175800092
:10ac6800c0758000010001000080fa004f03be009b
:10ac78004f02be004f01be004f00be003600f90073
:10ac880000400600801f78000200fa0034c0bf00b0
:10ac98000080fb00000f78000000200000407800d2
:10aca80034e0b7008660a90010c0b300eaf0b7002e
:10acb8001e0078000040780034e0b7000080fa00f9
:10acc8004f007800004006000a00fa00400798008c
:10acd800100280004500de00674060000080fb0035
:10ace800300798009002800010079800ff3ffc0092
:10acf80011028000000e2000008070001002880001
:10ad08001e0090009002880000008800e07f80000c
:10ad1800100f7800e07f800090007800300020005d
:10ad2800808f50000f003a00be009000000e2000f7
:10ad380080806000000e2000808f500004003a00e0
:10ad4800e07f80008000eb000108780003003700f6
:10ad5800e07f80001100200001087800e07f80007b
:10ad6800100f7800e07f8000900078004e0090007f
:10ad7800808f5000140032004e0090008000eb00dd
:10ad8800810f50000400320011002000810f500094
:10ad9800070032000c0037007000200030079800d0
:10ada800e07f8000ce0090000108780006003700a0
:10adb8000000eb0030079800e07f8000ce00900094
:10adc8000108780000000000900280002007980029
:10add800ff3ffc003e0090000040780067406000a4
:10ade8000080fb00670060004500dd001202800063
:10adf800f1f12f00810061000080700010028800ce
:10ae08002e00900090028800000088001e00780044
:08ae18000080fa0000000600b2
:020000040000fa
:10ae2000f40f00000a00000000000000fe0f000008
:10ae300002000000020000000000000000400000ce
:10ae40000008000000000000ea10000004000000fc
:10ae5000020000000000000000000000f6100000ea
:10ae60000200000000000000b40e00000a01000013
:10ae700000000000c81000002200000000000000d8
:10ae8000500800006406000000000000ee10000002
:10ae900004000000020000000000000000000000ac
:10aea000f810000002000000000000002010000068
:10aeb000a8000000000000000010000020000000ba
:10aec00000000000f210000004000000000000007c
:10aed000be0f00003600000000000000000000006f
:020000040000fa
:10aee00091018800800078000000eb001500370019
:10aef000e280400032a0b4009101ba00e28040003c
:10af000032a0b4009102ba00e280400032a0b40046
:10af10000002eb00472bde00f507b200602ce100d9
:10af200004003a000059eb008301e900fdff3e00f8
:10af3000040037006128e100010032000082eb00cc
:10af4000040007001101ba000200e000e8ff3a0027
:10af5000000006003159ba008301e9000c003200fc
:10af60002159ba008301e900080032000400e00022
:10af700003003a00e280400032a0b400f5ff370041
:10af800011d9ba008301e900faff3a008100e80014
:10af9000e180400032a0b40000000600af0f2100a5
:10afa0000e9f21000e018800000000000c00070029
:10afb0000071250001002000c9ff070000002000eb
:10afc0000000e0000200320000000200000000006b
:10afd000860e0200000000000040da000000fe00c3
:10afe0004440a900400e20000000e00003003200b1
:10aff00000002000a00188004440a80000000600d6
:020000040000fa
:10b000000000fa008020a900ffff37000000fa00ce
:10b010008060a900ffff37000000fa008040a9000f
:10b02000ffff37000000fa008080a900ffff370013
:10b030000000fa008020a900ffff37000000fa009e
:10b040008060a900ffff37000000fa008040a900df
:10b05000ffff37000000fa008080a900ffff3700e3
:020000040000fa
:10b06000f03fb1000180b10006003500ee03090099
:10b0700000000000403fb1000180b100fbff3d0037
:10b080001000b000203fb000020035000080090031
:08b090000000000000000600b2
:00000001FF
